:100000000C94550E0C94720E0C94720E0C94720E8D
:100010000C94720E0C94720E0C94720E0C94720E60
:100020000C94720E0C94AF120C94720E0C94720E0F
:100030000C94720E0C94720E0C94720E0C94720E40
:100040000C94720E0C94AF0F0C944E2E0C94222E26
:100050000C94720E0C94720E0C94720E0C94720E20
:100060000C94720E0C94720E0C94720E0C94720E10
:100070000C94720E0C94720E0C94720E0C94720E00
:100080000C94720E0C94720E0C94720EFD28992B27
:100090000829992B212921297A29BE29FD29482AB5
:1000A0008F29992B992BE02AF12A172B2C2B992B8E
:1000B000992B992B992B992B992B992B992B872B32
:1000C000992B992B992B692B6B2B702B3D2B992BF3
:1000D0007E2B322E312E3100696E636F6D7061742C
:1000E00069626C6520485700202025303258002076
:1000F000504300204C430045617379436F6E747226
:100100006F6C000102031718040506151107080992
:1001100016120A000B0C13100F0E0D14040E1F0EF6
:100120000E0E0E000E0E0E0E1F0E0400040E1F000B
:100130001F0E0400000404040010081300100B1329
:1001400000130B130001021900011A1900191A19E2
:10015000080C1E1F1E0C080002060F1F0F060200CF
:100160000E11111F1B1B1F001F0A0A0A0A0A1F007B
:100170001C101810160505050C17141714170C0081
:10018000040A110A0A0E00001C10181216020207B7
:100190001C101816110204071C1018161102010673
:1001A0001C1018151507010100000017151515176B
:1001B000121212121200000000000017111714177B
:1001C0001711131117000000000000151517111169
:1001D0001714171117000000070505050505050789
:1001E0000707070707070707030509121418100078
:1001F00003070F1E1C18100000060912141209062E
:1002000000060917170906001F111F001F111F0004
:100210001F111F001F1F1F001F1F1F001F111F0086
:100220001F1F1F001F1F1F00040E1F04041F0E04AA
:10023000010101050D1F0C0411040A11111F110009
:10024000110E111111110E000A00111111110E00E1
:100250000E11111611111610001C1F1F1F13101064
:10026000001C13111D13101000181711191710106E
:10027000001F11111F101010206D332020200000CE
:10028000204D4D4920200000204D4D02202000002F
:1002900020444343202000002053544F50200000AE
:1002A00053484F52542100002048414C5420000034
:1002B00020202020202000002050524F4720000006
:1002C0005245534554200000202054504D2000003A
:1002D000555044415445000020202020002533641F
:1002E00000252D31312E31317300252D3564002547
:1002F000632F256320256300256300462530326483
:100300003D25630020200102202020202020200005
:100310002533640025336400252D3564002D2D2DF3
:100320002D2020004144523A20256C6420202020BA
:1003300020202020202000232D007E0E0E0E0E1BDC
:100340001B1C0E1B1B7E0E0E0E0E636F72746F2035
:1003500028312E356D73292000006C756E676F2073
:1003600028342E3032356D7329004D6F746F726FE3
:100370006C61000000000000000044434320202086
:10038000202000000000000000004D4D2000000073
:100390000000000000000000000044434300000093
:1003A00000000000000000000000706F73697469B5
:1003B000766120284D4D290000006E6567617469E3
:1003C00076612028444343290000303A206F666656
:1003D00020202020202020202000313A2054616954
:1003E0006C626974732020202000323A202B20494F
:1003F000644E6F74696679202000333A202B2041C7
:1004000063636573736F72792000526970726973E8
:1004100074696E6120202020200053616C76612079
:100420002020202020202020200052697072697333
:1004300074696E6120202020200053616C76612059
:100440002020202020202020200020737461746F41
:10045000206C61796F757420200020737461746F53
:10046000206C61796F7574202000636F72746F2047
:1004700028312E356D73292020006C6172676F2042
:1004800028342E3032356D7329004D6F746F726FC2
:100490006C61000000000000000044434320202065
:1004A000202000000000000000004D4D2000000052
:1004B0000000000000000000000044434300000072
:1004C00000000000000000000000706F7369746994
:1004D000766120284D4D290000006E6567617469C2
:1004E00076612028444343290000303A2044657354
:1004F000616374697661646F2000313A20546169E8
:100500006C626974732020202000323A202B20492D
:10051000644E6F74696679202000333A202B2041A5
:1005200063636573736F72792000526573746175CC
:100530007261722020202020200047756172646162
:1005400072202020202020202000526573746175C5
:100550007261722020202020200047756172646142
:100560007220202020202020200020457374616408
:100570006F204D617175657461002045737461640D
:100580006F204D617175657461004B75727A20281A
:10059000312E356D7329202000004C616E672028B4
:1005A000342E3032356D732900004D6F746F726FC9
:1005B0006C61000000000000000044434320202044
:1005C000202000000000000000004D4D2000000031
:1005D0000000000000000000000044434300000051
:1005E00000000000000000000000706F7369746973
:1005F0007620284D4D29000000006E656761746902
:1006000076202844434329000000303A2061757366
:1006100020202020202020202000313A2054616911
:100620006C626974732020202000323A202B20490C
:10063000644E6F74696679202000333A202B204184
:1006400063636573736F72792000416E6C616765D7
:100650006E7A757374616E642000416E6C616765BB
:100660006E7A757374616E64200057696564657293
:100670006865727374656C6C6E005370656963684D
:1006800065726E2020202020200020776965646537
:100690007268657273742E20200020737065696320
:1006A0006865726E20202020200073686F727420AD
:1006B00028312E356D73292000006C6F6E6720285D
:1006C000342E3032356D732900004D6F746F726FA8
:1006D0006C61000000000000000044434320202023
:1006E000202000000000000000004D4D2000000010
:1006F0000000000000000000000044434300000030
:1007000000000000000000000000706F7369746951
:10071000766520284D4D290000006E65676174697B
:1007200076652028444343290000303A206F6666EE
:1007300020202020202020202000313A20546169F0
:100740006C626974732020202000323A202B2049EB
:10075000644E6F74696679202000333A202B204163
:1007600063636573736F72792000526573746F727F
:100770006520202020202020200053617665202045
:1007800020202020202020202000526573746F72CA
:100790006520202020202020200053617665202025
:1007A00020202020202020202000206C61796F75DF
:1007B00074207374617475732000206C61796F7597
:1007C000742073746174757320005B756E6B6E6F4B
:1007D000776E207374617475735D00466F726D611E
:1007E000746F20696E636F6D70617400466F726D17
:1007F00061746F20696E636F6D702E2000696E6B7F
:100800006F6D7061742E20466F726D617400696E39
:10081000636F6D7061742E20466F726D6174005B42
:10082000756E6B6E6F776E206572726F725D002EE3
:100830002E20617474656E64657265202E2E200012
:10084000233D63616E63656C6C6100000000000015
:10085000002876756F746F2900000000000000000A
:1008600000002E2E63616E63656C6C617A696F6E39
:10087000652E00206572726F726500000000000036
:100880000000000020736F6C6F2044434321202040
:100890002020202000207072696D61207072656DCB
:1008A0006920474F20002A3D416E6E756C6C6100D7
:1008B000000000000000002070726F6772616D6DB3
:1008C000617A696F6E6520002D636F72746F2063AB
:1008D0006972637569746F2D00206E617469766F3B
:1008E0002028313A312920202000206C696E656172
:1008F00072652028323A31292020002070726F67FB
:100900007265737369766F20312020002070726FDA
:10091000677265737369766F2032202000204D6FF7
:10092000646F204143202020202020202000204DE3
:100930006F646F20444320202020202020200020AE
:100940004175746F53746570202020202020200092
:100950002A6C656767692000000000000000000045
:10096000002A7363726976690000000000000000CD
:1009700000002E2E20736372697474757261202ECC
:100980002E20002E2E2E206C657474757261202E20
:100990002E2E2000212121206572726F7265202188
:1009A0002121202000204F4B20202020202020200B
:1009B0002020202020002E2073616C7661746167F6
:1009C00067696F202E20002E2E2072697072697365
:1009D00074696E6F202E2000233D43616E63202AD0
:1009E0003D416E6E756C202000233D5369202A3DE9
:1009F000416E6E756C6C6120200020636F6E6669BD
:100A0000677572617A696F6E6520005350454E5468
:100A10004F00000000000000000000002A204E658A
:100A20007373756E205472656E6F202A0020636F99
:100A300072746F20636972637569746F20002A2A6B
:100A40002A2074696D65206F7574202A2A2A004156
:100A500063636573732E20202534642F253464006E
:100A6000436F6E6669677572617A696F6E65202083
:100A70000020636F6E6669677572617A696F6E6573
:100A800020002E2E2E20657370657265202E2E2E6E
:100A9000202000233D626F7272617200000000002E
:100AA000000000002873696E2046696368612900B0
:100AB00000000000002E2E2E20626F7272616E64A4
:100AC0006F202E2E2E002046616C6C6F00000000FF
:100AD0000000000000000020736F6C6F20706172D6
:100AE00061204443432120002022474F222070727E
:100AF000696D65726F202020002A3D43616E636539
:100B00006C6172000000000000002050726F67727C
:100B1000616D6163696F6E202020002D636F7274B8
:100B20006F20636972637569746F2D00206E617444
:100B300069766F2028313A312920202000206C6905
:100B40006E6561722028323A312920202000207001
:100B5000726F677265737369766F20312020002091
:100B600070726F677265737369766F203220200030
:100B7000204D6F646F204143202020202020202022
:100B800000204D6F646F204443202020202020202F
:100B90002000204175746F53746570202020202040
:100BA0002020002A6C656572200000000000000013
:100BB000000000002A6573637269000000000000F5
:100BC00000000000002E2065736372696269656E23
:100BD000646F202E20002E2E2E206C6579656E64A9
:100BE0006F202E2E2E20002121212046616C6C6F5B
:100BF0002021212120202000204F4B2020202020B8
:100C00002020202020202020002E2E2067756172B9
:100C100064616E646F202E2E20002E207265737426
:100C2000617572616E646F202E2000233D426F72E9
:100C30007261202A3D43616E632E2000233D53697B
:100C4000202A3D43616E63656C6172200020436F12
:100C50006E66696775726163696F6E202000446516
:100C60007361637469766164612020202020002A0A
:100C70002A2A2053696E205472656E202A2A2A007F
:100C80002A636F72746F20636972637569746F2A67
:100C9000005469656D706F20657870697261646F6A
:100CA000200041636365732E202534642F2534644E
:100CB000000000436F6E66696775726163696F6EED
:100CC0002020200020436F6E66696775726163693A
:100CD0006F6E2020002E2E2E2077617274656E209C
:100CE0002E2E2E202000233D4CF6736368656E0087
:100CF00000000000000000286B65696E2045696EE9
:100D00007472616729000000202E2E2E206CF6736D
:100D1000636865202E2E2E2000204665686C657263
:100D200000000000000000000000206E75722066C8
:100D3000FC722044434321202020002065727374FC
:100D400020474F206472FC636B656E002A3D416250
:100D5000627275636800000000000000002050729D
:100D60006F6772616D6D696572756E6700002D2D1C
:100D7000204B75727A7363686C75DF202D2D00200F
:100D80004E617469762028313A31292020202000D4
:100D9000204C696E6561722028323A31292020206A
:100DA000002050726F67726573736976203120205E
:100DB00020002050726F677265737369762032204D
:100DC000202000204143204D6F6475732020202097
:100DD00020202000204443204D6F64757320202084
:100DE0002020202000204175746F537465702020EE
:100DF0002020202020002A6C6573656E0000000012
:100E0000000000000000002A736368722E000000DA
:100E100000000000000000002E2E20736368726541
:100E20006962656E202E2E00002E2E2E206C6573BA
:100E3000656E202E2E2E20200000212121204665C7
:100E4000686C657220212121200000204F4B20205A
:100E50002020202020202020202000002E2E207363
:100E6000706569636865726E202E2E000077696573
:100E70006465726865727374656C6C656E00233DA1
:100E80004CF6736368656E202A3D416262720023EE
:100E90003D4A61202A3D416262727563680000002C
:100EA000206CF6736368656E2020202020202020AF
:100EB0000041555300000000000000000000000049
:100EC00000002A2A206B65696E65204C6F6B202A12
:100ED0002A20002A2A204B75727A7363686C75DFAA
:100EE000202A2A002A205A656974FC62657273639D
:100EF00068722E2A00576569636865202534642F5F
:100F00002534640000004B6F6E666967757261740A
:100F1000696F6E20202000204B6F6E6669677572C6
:100F20006174696F6E2020002E2E2E207761697407
:100F3000696E67202E2E2E2000233D64656C65743B
:100F400065000000000000000000286E6F20656E44
:100F500074727929000000000000002E2E2E2064FB
:100F6000656C6574696E67202E2E2E002066617593
:100F70006C740000000000000000000000204443EA
:100F800043206F6E6C7921202020202020002070CB
:100F90007265737320474F20666972737400002A6C
:100FA0003D43616E63656C000000000000000000BE
:100FB0002070726F6772616D696E670000000000DB
:100FC000002D73686F727420636972637569742D84
:100FD0002000206E61746976652028313A3129201D
:100FE000202000206C696E6561722028323A312918
:100FF000202020002070726F6772657373697665B8
:1010000020312020002070726F67726573736976DB
:10101000652032202000204143204D6F6465202050
:1010200020202020202000204443204D6F64652094
:101030002020202020202000204175746F537465EB
:101040007020202020202020002A7265616420006A
:10105000000000000000000000002A77726974653B
:1010600000000000000000000000002E2E2E20775F
:10107000726974696E67202E2E2E20002E2E2E206F
:1010800072656164696E67202E2E2E200021212159
:10109000206661756C742021212120202000204FC2
:1010A0004B20202020202020202020202020002E27
:1010B0002E2E20736176696E67202E2E2E20200042
:1010C0002E2E20726573746F72696E67202E2E202B
:1010D00000233D44656C2E202A3D43616E63656CA0
:1010E0002000233D596573202A3D43616E63656C82
:1010F00020200020636F6E66696775726174696F86
:101100006E2020004F464600000000000000000056
:1011100000000000002A2A2A206E6F2054726169A4
:101120006E202A2A2A002A2073686F72742063694D
:10113000726375697420002A2A2A2074696D6520FB
:101140006F7574202A2A2A00506F696E742020253A
:1011500034642F253464000000436F6E6669677540
:10116000726174696F6E2020200020636F6E666963
:101170006775726174696F6E2020005B6E6F206D01
:101180006573736167655D004003A001CF00670070
:101190004400330019001000204D3320656E616259
:1011A0006C65642020202020003D253564003078C7
:1011B0002530386C580020253564002534646D7363
:1011C000002533642C25647300202E2E2E2E202023
:1011D00020202020202020002564206D7300202561
:1011E00032640025346400202D2D2D002020202085
:1011F00020202000204F4B20202020002533640099
:101200002D2D2D002534643A200025366400202D34
:101210002D2D2D2D0025346400202D2D2D0043561D
:101220003A253464204269743A25643D0043563AB5
:1012300020202020204269743A203D200025357569
:1012400000202D2D2D2D004142434445464748495D
:101250004A4B4C4D4E4F5051525354555657585976
:101260005A303132333435363738392E2C3A2D2B2B
:10127000232F3D3C7C3E20004D4D20492020313421
:1012800020004D4D20492020323761004D4D20492E
:101290002020323762004D4D2002202031342000C2
:1012A0004D4D20022020323761004D4D200220207C
:1012B000323762004443432020203134200044432D
:1012C000432020203238200044434320203132384C
:1012D00020006D3320202031323820003A200025B4
:1012E0003575005365724E722E2025386C750032AC
:1012F0002E312E3100536F6674772E205600253321
:1013000064004E723A202532642020004D656E75CF
:10131000204C6F636F6D6F746976650050726F67F4
:1013200072616D6D617A2E204443430050726F6785
:1013300072616D6D617A2E206D330000537461749B
:101340006F204C61796F757400000000496D706FFB
:1013500073746174696F6E65000000004C43442033
:10136000726574726F696C6C2E0000004C6F6B4379
:101370006F6E74726F6C000000000000557363693B
:1013800074610000000000000000000053656C65FF
:101390007A696F6E6120000000000000466F726D78
:1013A00061746F2044617469200000004E6F6D65A8
:1013B00020202020202000000000000056616C6FDB
:1013C00072652020202020000000000043562028C5
:1013D000627974652900000000000000435620284F
:1013E000626974290000000000000000496E642E4C
:1013F000205072696D6172696F000000496E642E41
:101400002045737465736F000000000052656769C2
:101410007374726F00000000000000005061676587
:101420002D4D6F6465000000000000004D61696E85
:1014300020547261636B0000000000005261696C0F
:10144000436F6D2043560000000000004D6F646F35
:101450002031323846530000000000004D6F646FA9
:10146000204A6F676469616C00000000496D706F0D
:101470007374617A2E2073383800000043616E6304
:10148000656C6C610000000000000000426F6F732B
:1014900074657200000000000000000056656C6F6B
:1014A0006369746120696E74657266004465632EB9
:1014B0004163636573736F7269000000466F726DFC
:1014C00061746F204C6F636F000000005061757392
:1014D00061207365676E2E4D4D200000537570704E
:1014E0006F72742E5261696C436F6D006D6F64751D
:1014F0006C69207338380000000000007465737454
:10150000206D6F64756C692073383800506F6C2ED5
:1015100020636F72746F636972632E0053656E731C
:101520002E20636F72746F6369722E005475747429
:1015300069206163636573736F726900466F726DD2
:101540002E206163636573736F7269006D696E2E1F
:10155000746D702E696D70756C736F006D61782E8F
:10156000746D702E696D70756C736F00696E64694F
:1015700072697A7A6F206D33000000004D656E75D8
:10158000204C6F636F6D6F746F72610050726F6784
:1015900072616D6D617220444343000050726F6749
:1015A00072616D6D6172206D33000000457374616E
:1015B000646F204D6171756574610000416A7573D7
:1015C000746573000000000000000000496C756D38
:1015D000696E6163696F6E204C4344004C6F6B43CE
:1015E0006F6E74726F6C00000000000053616C69D4
:1015F00072000000000000000000000053656C65F0
:101600006363696F6E61722000000000466F726D47
:1016100061746F204461746F730000004E6F6D62DF
:1016200072652020202000000000000046696368E9
:1016300061202020202000000000000043562028C8
:1016400062797465290000000000000043562028DC
:10165000626974290000000000000000446972659E
:101660006363696F6E20636F7274610044697265B1
:101670006363696F6E206C617267610052656769B0
:101680007374726F00000000000000005061676515
:101690002D4D6F646500000000000000456E20566F
:1016A0006961207072696E6369702E005261696CA5
:1016B000436F6D2043560000000000004D6F646FC3
:1016C00020313238207061736F7300004D6F646F8A
:1016D000206465206D616E646F000000416A75735F
:1016E000746573207338380000000000426F727216
:1016F000617200000000000000000000426F6F7384
:101700007465723A000000000000000041636365E8
:10171000736F72696F733A0000000000466F726D5C
:1017200061746F206465205472656E00506175733A
:1017300061205365F1616C204D4D00005375706F51
:10174000727465205261696C436F6D004D6F6475F2
:101750006C6F73207338380000000000507275659C
:101760006261204D6F642E2073383800506F6C2EEC
:1017700020436F72746F636972632E0053656E73DA
:101780002E20436F72746F6369726300546F646FCD
:10179000732041636365736F722E0000466F726D34
:1017A00061746F2061636365736F72004475726169
:1017B000632E496D70756C2E6D696E004475726193
:1017C000632E496D70756C2E6D6178004469726589
:1017D0006363696F6E206D33000000004C6F6B20F7
:1017E0004D656EFC00000000000000004443432DE6
:1017F00050726F6772616D6D672E00006D332050FF
:10180000726F6772616D6D672E000000416E6C61D2
:1018100067656E7A757374616E64000045696E73F6
:1018200074656C6C756E67656E0000004C434420F7
:1018300042656C6575636874756E67004C6F6B43C9
:101840006F6E74726F6C0000000000004578697460
:1018500000000000000000000000000041757377E8
:10186000E4686C656E20000000000000446174654F
:101870006E666F726D617400000000004E616D65F0
:1018800020202020202000000000000045696E7408
:1018900072616720202000000000000043562028CD
:1018A000627974652900000000000000435620287A
:1018B0006269742900000000000000004261736941
:1018C000732D416472657373650000006C616E670F
:1018D0006520416472657373650000005265676935
:1018E00073746572000000000000000050616765BD
:1018F0002D4D6F64650000000000000048617570A8
:1019000074676C6569730000000000005261696CC7
:10191000436F6D204356000000000000313238460E
:1019200053204D6F64650000000000005265676C35
:1019300065726D6F64757300000000007338382D98
:1019400045696E7374656C6C756E67004B6F6E667F
:10195000696775726174696F6E000000426F6F7322
:1019600074657200000000000000000057656963A4
:1019700068656E0000000000000000004C6F6B66A0
:101980006F726D6174000000000000004D4D2D531A
:1019900069676E616C205061757365005261696C96
:1019A000436F6D20537570706F7274007338382DEB
:1019B0004D6F64756C650000000000007338382DB1
:1019C0004D6F64756C746573740000004B75727AAA
:1019D0007363686C2E2D506F6C2E00004B75727AFD
:1019E0007363686C2E2D456D70662E00616C6C659E
:1019F000205765696368656E00000000576569637C
:101A000068656E666F726D61740000006D696E2EA0
:101A100020536368616C747A656974006D61782E17
:101A200020536368616C747A656974006D3320417A
:101A30006472657373650000000000004C6F636F93
:101A40006D6F74697665206D656E75004443432043
:101A500070726F6772616D6D696E67006D332070B3
:101A6000726F6772616D6D696E6700004C61796FAE
:101A70007574207374617475730000005365747419
:101A8000696E677300000000000000004C434420B2
:101A90006261636B6C696768740000004C6F6B4334
:101AA0006F6E74726F6C00000000000045786974FE
:101AB00000000000000000000000000053656C659D
:101AC00063742000000000000000000044617461A5
:101AD00020666F726D617400000000004E616D65DC
:101AE000202020202020000000000000456E74729D
:101AF00079202020202000000000000043562028EC
:101B00006279746529000000000000004356202817
:101B10006269742900000000000000005072696DC5
:101B200061727920616464726573730045787465CD
:101B30006E642E2061646472657373005265676918
:101B4000737465720000000000000000506167655A
:101B50002D4D6F6465000000000000004D61696E4E
:101B600020747261636B0000000000005261696CB8
:101B7000436F6D20435600000000000031323846AC
:101B800053204D6F64650000000000004A6F6764D9
:101B900069616C204D6F6465000000007338382067
:101BA00073657474696E67730000000044656C654A
:101BB000746500000000000000000000426F6F73B9
:101BC000746572000000000000000000506F696E34
:101BD0007473000000000000000000004C6F632ED2
:101BE00020666F726D617400000000004D4D20731F
:101BF00069676E616C207061757365005261696C14
:101C0000436F6D20537570706F7274007338382095
:101C10006D6F64756C6573000000000073383820C8
:101C20006D6F64756C6520746573740053686F72B2
:101C30007420632E20706F6C2E00000053686F724A
:101C40007420632E2073656E732E0000616C6C200F
:101C5000506F696E7473000000000000506F696E71
:101C6000747320666F726D61740000006D696E2E72
:101C70007377697463682E74696D65006D61782E81
:101C80007377697463682E74696D65006D332061C4
:101C9000646472657373000000000000202020302F
:101CA000782530386C582020200011241FBECFEF3B
:101CB000D0E1DEBFCDBF11E0A0E0B1E0ECEAFEE98B
:101CC00002C005900D92A03DB107D9F714E0A0ED38
:101CD000B1E001C01D92A238B107E1F70E94920E57
:101CE0000C94544F0C9400008091D001089581E031
:101CF0008093D101089580E00E94ED16BC018FEF22
:101D00006F3F780719F080E00E94FC2F0E948D271A
:101D10000E94C4198091D101882311F40E94891571
:101D2000A8950895CF93DF930E945C260E946E0FC2
:101D300083E068E04EE422E00E94E02D0E9438112A
:101D400078940E9461130E943725DC0114968C91CF
:101D50000E94841582E067EF70E00E94CF170E9416
:101D60004B25823021F00E944B25813021F482E006
:101D700063EF70E007C00E944B258038D9F482E001
:101D80006FEE70E00E94CF1781E060E00E940716BE
:101D900082E066E50E94FC1682E062ED70E00E943F
:101DA000CF170E943725EC0181E00E943714882369
:101DB00049F125C00E944B2500D000D00F92EDB70D
:101DC000FEB7319692E0ADB7BEB711969C9328EE60
:101DD00030E032832183838314820E9475170F9031
:101DE0000F900F900F900F9081E060E00E94071617
:101DF00082E068ED70E00E94CF17A895FECF80E0EA
:101E00000E94432682E00E943714882319F084E060
:101E10000E94432683E00E943714882319F085E04E
:101E20000E94432684E00E943714882329F081E031
:101E30000E94432601C0A8950E94D8278823D9F381
:101E400089859A85009749F060E070E040E050E0B5
:101E50000E94492DBC01009711F46A817B818FEFAC
:101E60000E94EF2581E011C00E9441200E945B1476
:101E7000BFEF8F3F9B07C1F70E947B0E8091D1017E
:101E80008823A1F31092D10180E00E944A1BEECF7B
:101E90009091D001981701F19630F1F0953011F43E
:101EA0008630D1F48093D001853029F480E060E25F
:101EB00045E00E940A278091D001863029F480E015
:101EC00060E246E00E940A278091D0010E94BF2F65
:101ED00081E08093D101089580E008958FE78ABB67
:101EE0001BBA80E187BB18BA80EF84BB8FEF85BB3C
:101EF0008BEB81BB8CEC82BB82E082B987EF83B92C
:101F000087E78093610081EE8093620087E1809390
:101F1000640089E1809365000E941A12A89588E107
:101F200081BD8EE081BD0895DC019091D50189E0ED
:101F3000989FF0011124EF52FC4F90E08D91819316
:101F40009F5F9930D9F78091D5018F5F8093D5013C
:101F50008091D501843010F01092D50108951F9220
:101F60000F920FB60F9211241F932F933F934F930D
:101F70005F936F937F938F939F93AF93BF93EF93F1
:101F8000FF9380910001909101012FEF8F3F920705
:101F900061F0BB9A8FB9769B0BC0BB981092D401AD
:101FA0001092DA011092D90103C0BB988FEF8FB95C
:101FB0001FB117FF8AC08091DB019091DC01892B52
:101FC000E1F08091D7018F5F8093D7018091D70195
:101FD000803210F01092D7019091D7018091D801F2
:101FE000981759F48091D8018F5F8093D801809120
:101FF000D801803210F01092D8018091D9019091CF
:10200000DA01815D934061F058F08091D6018F5FD5
:102010008093D6018091D601843010F01092D601C1
:102020001092DC011092DB011092DA011092D901BA
:1020300080910201181721F481E08093D40177C0C8
:102040001092D401412F50E04F775070682F70E00C
:102050004617570729F01F3F19F08F3F09F067C057
:102060008091D70129E0829FC00111248F549D4F98
:102070009093DC018093DB014617570709F057C0A6
:102080009091D5018091D601981721F488EA92E0C9
:102090000E94940F8091D60129E0829FC0011124F3
:1020A0008F529C4F9093DA018093D9018091D60191
:1020B0008F5F8093D6018091D601843010F010920A
:1020C000D60189E08093D20132C02091D401213021
:1020D00029F0213060F1263050F515C082E0809360
:1020E000D401103419F41092D30121C0113419F421
:1020F0002093D3011CC0123419F0133491F483E0FF
:102100008093D30114C0E22FF0E08091D30190E0DE
:1021100002968E179F0744F0E552FE4F80811817F4
:1021200019F01092D40103C02F5F2093D401809145
:10213000D401882329F0109300011092010121C0DD
:10214000E091D901F091DA013097A9F08191809363
:10215000000110920101F093DA01E093D90180911E
:10216000D20181508093D201882359F41092DA0170
:102170001092D90106C08FEF9FEF909301018093D9
:102180000001E091DB01F091DC01309749F083E040
:10219000E13DF80728F41193F093DC01E093DB01B3
:1021A000FF91EF91BF91AF919F918F917F916F912F
:1021B0005F914F913F912F911F910F900FBE0F9004
:1021C0001F9018951F93AC011FB7F8942091D5016B
:1021D0008091D60130E090E001972817390741F04F
:1021E0008091D501833039F48091D601882319F488
:1021F0001FBF80E005C0CA010E94940F1FBF81E08D
:102200001F910895DC01E8EAF2E08D91819382E06C
:10221000E13BF807D1F708959C01009739F14FB7DA
:10222000F8949091D7018091D801981721F44FBF6D
:1022300020E030E01BC09091D80189E0989FF00128
:102240001124EF54FD4FD90190E081918D939F5F50
:102250009930D9F78091D8018F5F8093D801809110
:10226000D801803210F01092D8014FBFC9010895F3
:102270000E944125262F2F772093E00147E0969575
:102280008795779567954A95D1F7262F2F772093D5
:10229000DF0137E096958795779567953A95D1F761
:1022A000262F2F772093DE0127E096958795779547
:1022B00067952A95D1F76F776093DD0187B3807FAB
:1022C00087BB88B3807F88BB84EE8DB9089588234F
:1022D00051F08091650084608093650000000000EB
:1022E000000000000895809165008B7F8093650059
:1022F00008950F931F93DF93CF930F92CDB7DEB75F
:10230000182F8AB3807F8ABB80E00E94671180917A
:102310006500826080936500112321F08091650043
:10232000816003C0809165008E7F8093650000000E
:10233000000081E00E94671109B380E00E946711EC
:1023400010E084E0000F111F8A95E1F70000000003
:102350000000000081E00E94671199B39F70902BEC
:1023600080E099830E9467118AB38F608ABB99814C
:10237000892F0F90CF91DF911F910F91089580E0E9
:102380000E947911982F87FF11C08091E4019091EC
:10239000E50128E08130920714F080E0089501966D
:1023A0009093E5018093E40181E008958091E60136
:1023B000882319F49F779093E7011092E50110921A
:1023C000E40180E008959B01AC018091F7039091B6
:1023D000F803A091F903B091FA0382179307A407B9
:1023E000B50798F08091F7039091F803A091F90355
:1023F000B091FA0360E0821B930BA40BB50B8050E5
:102400009041A040B040A0F412C08091F703909199
:10241000F803A091F903B091FA0360E0281B390B8F
:102420004A0B5B0B2050304F4F4F5F4F08F061E07D
:10243000862F089510927D0080B7877F80BF17BEDA
:1024400011BE89E683BF8BE085BD8FE183BD87B771
:10245000806887BF0895EF92FF920F931F9320919A
:10246000F7033091F8034091F9035091FA037C018E
:1024700000E010E0E20EF31E041F151F01C0A89536
:10248000C801B7010E94E3118823C9F31F910F917E
:10249000FF90EF900895FF920F931F93082F162F30
:1024A000F42E809165008D7F8093650080E00E940E
:1024B00067118AB38F608ABB8BB3902F92959F7000
:1024C000807F982B9BBB112321F080916500816058
:1024D00003C0809165008E7F8093650081E00E943B
:1024E000671180E00E946711FF2029F088E090E0EA
:1024F0000E942B120FC08BB30F70807F802B8BBB81
:10250000000000000000000081E00E94671180E0F0
:102510000E9467111F910F91FF900895EF92FF9213
:102520000F931F932091F7033091F8034091F90323
:102530005091FA037C0100E010E0E20EF31E041F4C
:10254000151F02C00E947B0EC801B7010E94E31153
:102550008823C1F31F910F91FF90EF9008951F9270
:102560000F920FB60F9211241F932F933F934F9307
:102570005F936F937F938F939F93AF93BF93EF93EB
:10258000FF938091E101882309F089C081E0809365
:10259000E10178948091E3018F5F8093E301809162
:1025A000E30190E083709070009719F0019741F576
:1025B00016C08091F7039091F803A091F903B091B0
:1025C000FA030196A11DB11D8093F7039093F803C0
:1025D000A093F903B093FA030E94431411C08091B1
:1025E000F7039091F803A091F903B091FA03817079
:1025F0009070892B19F00E94751402C00E94FB1381
:102600008091E201882321F00E94BF118093E201B2
:102610008091E201882309F040C09091FB038091F2
:10262000FC039817B9F18091FC03E82FF0E0E55026
:10263000FC4F9281182F1F5F103108F010E0903886
:1026400001F58091FB03811729F1E12FF0E0E550BE
:10265000FC4F92819F3F19F49091E701906897FF9A
:1026600002C01092E601892F807C803419F481E049
:102670008093E6011F5F103108F010E0892F60E0C1
:1026800002C0892F61E040E00E944B121093FC03CE
:1026900081E001C080E08093E2011092E101FF91AE
:1026A000EF91BF91AF919F918F917F916F915F91CA
:1026B0004F913F912F911F910F900FBE0F901F9040
:1026C0001895CF93DF9388E290E00E942B1280E36D
:1026D00060E041E00E944B1280E360E041E00E9434
:1026E0004B1280E360E041E00E944B1280E260E028
:1026F00041E00E944B1288E20E94F11580E40E94A2
:10270000F1158AE00E94C41589E20E94F1158CE15E
:102710000E94F11582E50E94F11589E60E94F115EB
:1027200084E70E94F11580E40E94F11585E10E9482
:10273000C41588E20E94F11580E40E94F1150E9400
:10274000F817EC0101C0A8959091FB038091FC0360
:102750009817C9F70E94BF118823A9F781E00E944A
:1027600079118A3019F481E089AB01C019AA88E097
:102770000E94F11581E00E94F11586E00E94F1159A
:102780008CE00E94F11580E060E00E94071680E076
:102790006CE171E00E94E81681E060E671E00E9461
:1027A000E81682E068E671E00E94E81683E068E7D8
:1027B00071E00E94E816DF91CF9108959091EA01AF
:1027C000E92FF0E0E651FE4F82839F5F9093EA018C
:1027D000983010F01092EA019091EB018091EA019B
:1027E000981741F4892F8F5F8093EB01883010F0A8
:1027F0001092EB01089531B12091E901220F36FDCD
:102800002160822F83708150823028F424FF02C01F
:102810002E6001C0217F2093E9019091E801990F7A
:1028200037FD9160892F83708150823028F494FFA6
:1028300002C09E6001C0917F9093E801207C892FA7
:10284000807C203831F4882341F0803C79F48AE19F
:1028500005C0203459F4803C21F489E10E94DE1344
:102860000895882319F48AE10E94DE1308958931BE
:1028700010F080E00895E82FF0E0EC50FE4F8081EA
:10288000811181E0089530912602343029F485B316
:10289000806F85BB97980895979A25B380E190E063
:1028A00002C0880F991F3A95E2F78095807F2F70BC
:1028B000822B85BB08959091EB018091EA018917E5
:1028C00019F42FEF3FEF0FC0E92FF0E0E651FE4F74
:1028D0008281282F30E0892F8F5F8093EB01883031
:1028E00010F01092EB01C90108958F929F92AF9260
:1028F000BF92CF92DF92EF92FF920F931F93CF93ED
:10290000DF930E94740E982F80912702981729F068
:102910009093270282E20E94DE1383B3E1B0EE0CB3
:10292000EE0C90E1E9228F70E82ACC24DD2495E0BA
:10293000892E81E0A82EB12C99249394E09126024F
:10294000E89DF0011124EC0DFD1DED5FFE4FF490AC
:1029500088E18F1508F481C00E2D0A250170CF2D56
:10296000D0E0FE01E35FFD4F1081110F0E944B2567
:10297000803819F4002371F009C001111160812F12
:1029800090E0817190708131910511F41F6103C055
:10299000892B09F4107E812F90E08076907080342E
:1029A000910519F41F7182E00CC08032910519F471
:1029B000106E81E006C08036910511F080E001C004
:1029C00083E0FE01E35FFD4F1083823099F0833096
:1029D00059F1813009F041C096E1F91621F4809156
:1029E0000902882319F48F2D0E94DE13CC50DE4F8C
:1029F000988233C0CC50DE4F18828F2D80680E94A1
:102A0000DE130E94740E853041F585E1F81619F445
:102A100080910A0205C096E1F916F9F48091090245
:102A20008823D9F486E017C0FE01EC50FE4F808168
:102A30008F5F8083882309F490828BEEF80E91E0FB
:102A40009F1558F080910902893738F080910A0269
:102A5000893718F085E00E94480F0894C11CD11CEA
:102A600085E0C816D10411F0E69468CF8091260263
:102A70008F5F80932602853010F010922602DF913E
:102A8000CF911F910F91FF90EF90DF90CF90BF906B
:102A9000AF909F908F90089590932804809327047F
:102AA000892B89F170932604609325048091F703A4
:102AB0009091F803A091F903B091FA039B0140E0D3
:102AC00050E0280F391F4A1F5B1F209321043093C9
:102AD00022044093230450932404809120048E7F89
:102AE00080932004211531054105510561F481E0F1
:102AF00090E0A0E0B0E08093210490932204A093A2
:102B00002304B09324040895813308F080E381BF47
:102B100008958091270490912804892BA1F1609158
:102B200021047091220480912304909124040E9436
:102B3000E311882341F180912004E0912704F09172
:102B40002804817009958091200491E08927809361
:102B500020042091F7033091F8034091F90350913C
:102B6000FA038091250490912604A0E0B0E0820F42
:102B7000931FA41FB51F8093210490932204A09358
:102B80002304B093240408951F93182F03C00E94B8
:102B90008D27A8952091FB038091FC0330E090E005
:102BA00001972817390799F38091FB038F3021F49F
:102BB0008091FC03882359F3F894E091FB03F0E043
:102BC000E550FC4F12838091FB038F5F8093FB03E2
:102BD0008091FB03803110F01092FB0378941F91D9
:102BE00008951F93182F80E80E94C415812F0E941A
:102BF000C4151F910895109228041092270481E0B3
:102C00000E94F11508958CE00E94F11508958295B7
:102C1000880F880F807C860F80680E94F1150895C8
:102C2000BF92CF92DF92EF92FF920F931F93CF93B9
:102C3000DF93C82EB62E8A01109228041092270422
:102C400021E02817A0F13FE0361788F14115510522
:102C500071F1FA0101900020E9F73197DE2ED41AC4
:102C600080E18D1510F490E1D92E8C2D6B2D0E94F2
:102C70000716E8018DE0E82E84E0F82E08C0888170
:102C8000F70181937F01699182E00E94FC169E0109
:102C9000201B2D15A0F3C0921D04B0921E04D092EB
:102CA0001F048AE896E164EF71E00E944C15DF9101
:102CB000CF911F910F91FF90EF90DF90CF90BF9039
:102CC0000895DF93CF93CDB7DEB7A0970FB6F894F2
:102CD000DEBF0FBECDBFDE0111969E01205E3F4FCD
:102CE00004C09D93A217B30731F0FA014F5F5F4F05
:102CF00094919923B1F71C92AE014F5F5F4F0E94F0
:102D00001016A0960FB6F894DEBF0FBECDBFCF91C0
:102D1000DF9108950F931F93CF93DF93082F809136
:102D20001D0460911E040E94071610E0CDE0D4E05F
:102D300009C0002311F460E201C0699182E00E94A1
:102D4000FC161F5F80911F04181798F3DF91CF9135
:102D50001F910F9108950E9407168EE00E94F115B1
:102D60000895EF92FF920F931F93CF93DF93382F25
:102D70007B01122F883028F5483018F5842F90E019
:102D8000820F911D099714F018E0141B330F330FB5
:102D9000330F340F832F80640E94F115C0E0D0E020
:102DA000012F10E008C0F701EC0FFD1FE4918E2FFA
:102DB0000E94C4152196C017D107ACF38FEF0E9473
:102DC000F115DF91CF911F910F91FF90EF90089532
:102DD00040E028E00E94B1160895882341F0833036
:102DE00019F02FEF3FEF06C00E945B1402C00E9453
:102DF0004A2F9C01C90108951F93162F882309F4B7
:102E00005EC0823009F05EC067FF55C00E94F817AF
:102E1000FC0181A98823E1F0143E11F414E84BC0B1
:102E2000163F11F414E947C01C3F11F411E843C0E8
:102E3000143C11F41EE83FC0163D11F419E93BC0E3
:102E40001C3D11F41AE937C0113F69F51BE933C085
:102E5000143E11F411EE2FC0163F11F41FEE2BC0DB
:102E60001C3F11F415EF27C0113F11F41EEE23C0D3
:102E7000143C39F484E068E372E00E94E81614E040
:102E80001AC0163D39F485E060E472E00E94E8164D
:102E900015E011C01C3D39F486E068E472E00E9440
:102EA000E81616E008C01F3D31F487E060E572E0E7
:102EB0000E94E81617E0812F0E94C41503C0862FD8
:102EC0000E941A2F1F9108951F93CF93DF93182FFD
:102ED000EB0104C02196812F0E94FC1668816623B5
:102EE000C9F7DF91CF911F9108950F931F93DF933F
:102EF000CF93CDB7DEB7C055D0400FB6F894DEBF44
:102F00000FBECDBF9E01265A3F4F8E010F5F1F4F50
:102F1000C8016A966EAD7FAD6A97A9010E945F4CA9
:102F200068968FAD6897B8010E946417C05BDF4F49
:102F30000FB6F894DEBF0FBECDBFCF91DF911F91CA
:102F40000F9108950F931F93DF93CF93CDB7DEB703
:102F5000C055D0400FB6F894DEBF0FBECDBF9E0166
:102F6000265A3F4F8E010F5F1F4FC8016A966EAD04
:102F70007FAD6A97A9010E94434C68968FAD689710
:102F8000B8010E946417C05BDF4F0FB6F894DEBF34
:102F90000FBECDBFCF91DF911F910F9108951F9369
:102FA000CF93DF93182FEB0104C0812F0E94FC16F2
:102FB0002196FE0164916623C1F7DF91CF911F91A5
:102FC0000895E82FF0E0EF70F070E65CFC4FE491BC
:102FD0008E2F90E0089590E083709070009731F00C
:102FE000039711F48CE1089584E008958FE108952A
:102FF0008DE292E008958091490282FF05C08091A0
:103000002F0290913002089580912D0290912E020E
:1030100008959091490291FD19C092FF05C08091D9
:103020002904823099F404C0809129048F3071F40E
:10303000109229049260977F9093490210924D025A
:1030400080E090E060E070E00E944C1508958823D5
:10305000E9F082E068EA71E00E94E81683E060EB44
:1030600071E00E94E81684E068EB71E00E94E816C7
:1030700085E060EC71E00E94E81686E068EC71E0A3
:103080000E94E81687E060ED71E01CC082E068E60F
:1030900071E00E94E81683E068E771E00E94E8169C
:1030A00084E068E871E00E94E81685E060E971E07C
:1030B0000E94E81686E068E971E00E94E81687E061
:1030C00060EA71E00E94E816089580912C02833036
:1030D00014F010922C0280912C028F5F80932C02AE
:1030E0008150813041F0823061F0882379F481E0B1
:1030F00060E772E003C081E068E672E00E94E816D3
:10310000089581E060E672E00E94E8160895882341
:1031100021F082E060EF71E003C082E068EE71E0D0
:103120000E94E8160895882321F081E060EE71E0A6
:1031300003C081E068ED71E00E94E8160895FF92F7
:103140000F931F93DF93CF9300D000D000D0CDB763
:10315000DEB78C01F62EFE01319686E0DF011D926E
:103160008A95E9F7D8016D917C91CF010E949E2646
:10317000F801808D918DA28DB38D282F2F772B8311
:1031800037E0B595A795979587953A95D1F7282F6C
:103190002F772C8327E0B595A795979587952A9546
:1031A000D1F781708D83FF2011F080648D8380E0E2
:1031B0006BE1AE014F5F5F4F0E94F42626960FB67B
:1031C000F894DEBF0FBECDBFCF91DF911F910F915D
:1031D000FF90089580935D020E94770E08952091DC
:1031E000490221FD0EC02B7F21602093490290935C
:1031F000300280932F0270933802609337020E944E
:10320000770E0895E0912D02F0912E028E179F0700
:1032100011F0EF2BF1F49B0140E050E0A9013327BE
:1032200022278091330290913402A0913502B0910F
:103230003602A070B070282B392B4A2B5B2B2093C1
:1032400033023093340240933502509336020E9489
:10325000770E0895FC0180912D0290912E02E817BF
:10326000F90711F510924C0260934B0260E070E098
:103270008091330290913402A0913502B0913602D0
:1032800080709070482B592B6A2B7B2B222311F0D6
:10329000616001C06E7F40933302509334026093AB
:1032A0003502709336020FC080912F029091300248
:1032B000E817F90751F410924C0260934B025093B7
:1032C0003802409337020E94770E08951F93182FFB
:1032D00080E06CE00E940716112309F100D000D0B5
:1032E0000F92EDB7FEB7319682E0ADB7BEB711963B
:1032F0008C938DED92E09283818380914D0290E0DA
:103300008F779070948383830E9475170F900F902E
:103310000F900F900F9080E00E94C41505C082E0CE
:1033200068ED72E00E94CF171F910895EF92FF920F
:103330000F931F93182F80FF02C083E001C085EA1E
:103340000E94C415E12E11FF02C084E001C085EA8D
:103350000E94C415E2FE02C085E001C085EA0E9419
:10336000C415E3FE02C086E001C085EA0E94C415D0
:10337000E4FE02C087E001C085EA0E94C4151F91E7
:103380000F91FF90EF9008956091390270913A0289
:1033900080913B0290913C02611571058105910578
:1033A00061F00E94E311882341F0109239021092DB
:1033B0003A0210923B0210923C0260913D027091E1
:1033C0003E0280913F029091400261157105810596
:1033D000910571F00E94E311882351F010923D0293
:1033E00010923E0210923F02109240020E94770E0D
:1033F0006091410270914202809143029091440297
:10340000611571058105910561F00E94E311882322
:1034100041F0109241021092420210924302109227
:10342000440280914C0218166CF420914B0230E05B
:103430002F77307080914E0290E02817390714F0F2
:1034400010924C0280914C0287FF09C080914B0280
:1034500090E08F779070892B11F410924C0280913C
:103460004C02209128023091290240912A02509169
:103470002B02882381F4211531054105510511F0F6
:103480000E94770E109228021092290210922A02AE
:1034900010922B020895211531054105510539F08F
:1034A000CA01B9010E94E311882309F46CC080911C
:1034B0004C02181644F40E94740E833049F4809133
:1034C0004B028F5F03C080914B02815080934B026F
:1034D00080914C02813059F08F3F49F0823061F089
:1034E0008E3F51F028E833E140E050E009C020E38E
:1034F00035E740E050E004C020EE3EE240E050E01E
:1035000080914E028E3781F48091F7039091F803F9
:10351000A091F903B091FA03F7E0569547953795D6
:103520002795FA95D1F721C08E3081F48091F70369
:103530009091F803A091F903B091FA03E4E0569555
:10354000479537952795EA95D1F70FC08091F703F6
:103550009091F803A091F903B091FA0375E05695A4
:103560004795379527957A95D1F7280F391F4A1F28
:103570005B1F209328023093290240932A02509324
:103580002B020E94770E08958091490280FD25C08C
:103590006091390270913A0280913B0290913C0215
:1035A000611571058105910521F00E94E3118823C1
:1035B000A1F01092300210922F021092500210923D
:1035C0004F0210922E0210922D0210924902109278
:1035D00051020E94770E81E0089580E008951F93C4
:1035E000FC01009769F4109249021092390210927E
:1035F0003A0210923B0210923C020E94C41A48C048
:103600007091490271FD44C060934B02CA01A0E071
:10361000B0E0209133023091340240913502509154
:10362000360220703070822B932BA42BB52B809305
:10363000330290933402A0933502B0933602809106
:10364000F7039091F803A091F903B091FA03885120
:103650009C4FAF4FBF4F81608093390290933A02E5
:10366000A0933B02B0933C0272FF09C071607B7F64
:1036700070934902F0933002E0932F0207C07E7FDF
:1036800070934902F0932E02E0932D020E94770E70
:103690001F910895DF92EF92FF920F931F93109165
:1036A0005D02112399F081E060E00E940716812FEE
:1036B00081500E94EA24BC0182E00E94CF17109240
:1036C0005D0288EE93E00E948E1202C0882319F0FA
:1036D0000E94FB1504C080E060E00E940716809104
:1036E0002D0290912E02892BF9F00E943725FC01C2
:1036F00040912D0250912E0282819381841795076B
:1037000049F42185328580914F029091500228170B
:10371000390751F05383428380914F0290915002B8
:10372000928781870E941A2620912D0230912E02C5
:1037300021153105C9F4109233021092340210920F
:1037400035021092360210924C02109238021092FA
:10375000370210924B0210924D02809149028F7EE7
:103760008093490210924A028091490282FD0DC065
:103770008091450290914602A0914702B091480283
:103780000097A105B10531F430C082E067E373E032
:103790000E94CF178DB79EB707970FB6F8949EBFBC
:1037A0000FBE8DBFEDB7FEB7319682E0ADB7BEB7A5
:1037B00011968C9384E293E09283818380914502F9
:1037C00090914602A0914702B0914802838394836E
:1037D000A583B6830E947517EDB7FEB737960FB66F
:1037E000F894FEBF0FBEEDBF51C02115310531F475
:1037F00082E06DE173E00E94CF1721C000D000D0BD
:103800000F92EDB7FEB7319682E0ADB7BEB7119615
:103810008C9388E193E092838183348323830E9495
:103820007517809149020F900F900F900F900F9095
:1038300080FF02C081E001C080E20E94C4151091A7
:103840004A020E94740E682F863008F0615063307F
:1038500091F480912D0290912E02892B61F0612FBD
:1038600070E06370707003E0660F771F0A95E1F7F0
:1038700068587D4F08C070E013E0660F771F1A95F7
:10388000E1F768567D4F82E00E94CF1780E06CE040
:103890000E9407168091490283FF12C000D000D019
:1038A0000F92EDB7FEB7319682E0ADB7BEB7119675
:1038B0008C9384E193E09283818380914D0211C0C7
:1038C00000D000D00F92EDB7FEB7319682E0ADB7D1
:1038D000BEB711968C9380E193E0928381838091AF
:1038E0004B0290E08F779070948383830E947517CA
:1038F0000F900F900F900F900F9080912D0290914C
:103900002E02892B89F080914A028370813081F4E4
:1039100087E10E943714882339F080E00E94C415A3
:1039200080E068E272E05BC080E20E94C41559C08A
:1039300080E00E94C4150E943725FC01808185FF2C
:1039400043C080914B0287FF04C080E06CE271E0CD
:1039500003C080E060E371E040E024E00E94B11623
:1039600080914C028823E1F018163CF08E3F81F0E4
:103970008F3F94F48D3FA9F507C08230C9F08230A3
:103980009CF0833071F518C080E06CE471E017C0E2
:1039900080E068E471E013C080E064E471E00FC08F
:1039A00080E064E371E00BC080E068E371E007C091
:1039B00080E06CE371E003C080E060E471E044E02B
:1039C00024E00E94B1160DC080914B0287FF04C015
:1039D00080E06CE171E003C080E064E271E00E948D
:1039E000E8160E94740E813049F489E00E94072590
:1039F000AC0181E060E00E94611603C2809149023F
:103A000083FD06C080E060E040E050E00E941016B8
:103A10008091490287FD03C000E010E014C080914E
:103A20002F0290913002892B19F001E010E00BC0B9
:103A300080914A020E94EB1720E030E0853010F0C0
:103A400021E030E08901F02E81E060E00E9407165D
:103A50008091450290914602A0914702B0914802A0
:103A60000097A105B10509F429C18DE00E94371422
:103A7000882329F48EE00E943714882381F100D036
:103A80000F9282E0EDB7FEB7818384E093E09383E9
:103A900082830E9475170F900F900F908DE00E9407
:103AA0003714882369F081E060EE71E00E94E81627
:103AB00082E068EE71E00E94E81683E998E10CC0AC
:103AC00081E068ED71E00E94E81682E060EF71E04D
:103AD0000E94E81687E898E16CE271E0ECC087E0AC
:103AE0000E940725BC0182E00E94CF1787E00E9458
:103AF00007250E94234C182F04C080E20E94C415A1
:103B00001F5F1031D0F310914A02812F0E94EB17F2
:103B100090E0A0E0B0E02091450230914602409153
:103B200047025091480282179307A407B5070CF487
:103B30004DC081E06BE00E940716609145027091D4
:103B4000460281E090E0A0E0B0E0062E04C0880FBD
:103B5000991FAA1FBB1F0A94D2F7209133023091FC
:103B60003402409135025091360282239323A423DC
:103B7000B5230097A105B10519F425EA30E002C08C
:103B800023E030E08DB79EB707970FB6F8949EBF3D
:103B90000FBE8DBFEDB7FEB7319682E0ADB7BEB7B1
:103BA00011968C938BEF92E092838183CB01638398
:103BB0009483368325830E947517EDB7FEB7379639
:103BC0000FB6F894FEBF0FBEEDBFC0C01370133028
:103BD00009F0BCC08FE00E943714882351F480E1C3
:103BE0000E943714882329F48CE00E94371488231C
:103BF00069F180E10E943714882321F081E060E6BA
:103C000072E003C081E068E572E00E94E81681E09E
:103C10006FE00E94071600D000D00F92EDB7FEB7FC
:103C2000319682E0ADB7BEB711968C9388EF92E0E3
:103C30009283818381E090E0948383830E9475174F
:103C40000F900F900F900F900F90DBC081E060E617
:103C500072E00E94E81681E06BE00E940716EDB763
:103C6000FEB739970FB6F894FEBF0FBEEDBF319681
:103C700082E0ADB7BEB711968C938FEE92E092833F
:103C8000818386E090E09483838387E090E096834D
:103C9000858381E090E0908787830E947517EDB758
:103CA000FEB739960FB6F894FEBF0FBEEDBF85E69E
:103CB00098E168EC70E00E944C15A3C020912F029F
:103CC000309130022115310539F100D000D00F922A
:103CD000EDB7FEB7319682E0ADB7BEB711968C93C3
:103CE0008AEE92E092838183348323830E94751746
:103CF0000F900F900F900F900F90809137028F715F
:103D00000E949619002321F08CE30E94C4152DC057
:103D100080E20E94C4151CC000D000D00F92EDB705
:103D2000FEB7319682E0ADB7BEB711968C9381EEA7
:103D300092E09283818381E592E0948383830E9461
:103D400075170F900F900F900F900F90FF2069F450
:103D500080913D0290913E02A0913F02B0914002BD
:103D60000097A105B10509F444C080912F029091FC
:103D70003002892BF1F580914A020E94EB178530C1
:103D8000C0F181E060E00E94071686E40E94C4153D
:103D9000DD24D394B2E0EB2EF12C012D112D809176
:103DA000330290913402A0913502B09136028E21F7
:103DB0009F21A023B1230097A105B10549F0B9E0E7
:103DC000BD1518F08D2D805D04C08D2D885001C06B
:103DD00085EA0E94C415D394E0E1DE1629F0EE0CCA
:103DE000FF1C001F111FDBCF80E20E94C41581E081
:103DF00006C0809133028F710E94961980E00E9464
:103E000027181F910F91FF90EF90DF900895CF93A7
:103E1000DF93EB0180934A02E82FF0E0EF70F0703F
:103E2000E65CFC4FE491E0934E026115710559F098
:103E3000CB0160E070E041E552E00E94492DD09353
:103E40005002C0934F020E94770EDF91CF910895E8
:103E5000AC01809149028C7F8093490210925002FC
:103E600010924F02662309F045C010925102209132
:103E70002D0230912E022115310521F030933202AE
:103E800020933102109233021092340210923502C4
:103E900010923602109238021092370210923002BD
:103EA00010922F0210922E0210922D0210924C02AC
:103EB00010924A02109229044115510551F18FEFD9
:103EC000BA010E94EF258091490281FD22C0109223
:103ED0003302109234021092350210923602109280
:103EE000300210922F0210922E0210922D02109288
:103EF0004A020DC01092290460912D0270912E0289
:103F00008FEF0E94B6258091490281FD02C090E0AA
:103F100001C091E0809149028B7F826080934902C9
:103F2000892F0895EF92FF920F931F93DF93CF9302
:103F300000D000D000D0CDB7DEB77C01FE013196B5
:103F400086E0DF011D928A95E9F7F701208D318D1A
:103F5000428D538D2030F8E23F07F0E04F07F0E04C
:103F60005F072CF0D7015C968C9186FF7DC02030D6
:103F7000B0E43B07B0E04B07B0E05B070CF074C067
:103F8000F70162817381211531054105510509F45D
:103F90005DC06115710559F180819181A0E0B0E0AB
:103FA00082179307A407B50741F0CB01A0E0B0E06A
:103FB00082179307A407B507D1F4D7015C968C91BB
:103FC0005C978E7F5C968C935C976D917C918E0153
:103FD0000F5F1F4FC8010E949E2680E065E0A80188
:103FE0000E94F426F7011382128211821082D701F7
:103FF0008D919C91A0E0B0E0F701208D318D428D34
:10400000538D82179307A407B50769F4848D91E057
:1040100089278B7F848FD70158961D921D921D9200
:104020001C925B9721C081E060E00E94071680E04F
:104030000E940725BC0182E00E94CF17F701648D22
:104040006470808D918D0E94281F09C0672B39F400
:10405000D7015C968C915C9784605C968C93F70199
:10406000108E118E128E138E26960FB6F894DEBF28
:104070000FBECDBFCF91DF911F910F91FF90EF90B9
:104080000895AF92BF92DF92EF92FF920F931F932A
:10409000DF93CF93CDB7DEB72C970FB6F894DEBF82
:1040A0000FBECDBF9C015E010894A11CB11C86E02F
:1040B000D5011D928A95E9F72531310509F49AC396
:1040C000263131052CF52C30310509F47DC12D3018
:1040D0003105ACF42A3031054CF4213031050CF0B7
:1040E000E3C32115310509F493C328C42A303105EF
:1040F00009F40CC42B30310509F020C4FEC3213172
:1041000031050CF0A2C22F3031050CF00DC333C2C3
:104110002A38310509F4F6C32B383105A4F42B31C4
:10412000310564F4293131051CF52631310509F4D6
:104130001BC32731310509F001C40BC123323105FE
:1041400009F0FCC3F2C32F3831054CF42D3831058A
:104150000CF011C22C38310509F0F0C3E9C1213946
:1041600031050CF4FBC22739310509F0E7C3E4C37C
:104170008091490283FF03C010914D0202C010914B
:104180004B0200E02931310509F401E0E0904E02D4
:104190000E943725FC01F7800E943725FC018081B1
:1041A00084FF35C017FD05C080E0002309F481E0DD
:1041B000082F002311F001E02CC0812F90E08F77B1
:1041C0009070892B79F48091410290914202A091E4
:1041D0004302B09144020097A105B10519F4212FC3
:1041E0002058ADC08091F7039091F803A091F90396
:1041F000B091FA03845D9E4FAF4FBF4F8093410251
:1042000090934202A0934302B093440224C000233F
:1042100011F10E943725FC01808185FF07C0809144
:104220004C0283300CF08AC08F5F21C00E94740E54
:10423000833009F083C0812F90E08F7790702E2D0E
:1042400030E0821793070CF079C0FEE7EF16E1F536
:10425000FF20E1F439C00E943725FC01808185FFF1
:1042600009C080914C028E3F0CF468C0815080934D
:104270004C0264C0812F90E08F779070892B09F4F5
:104280005DC04EE7E41641F5FF2031F181E0F816FC
:1042900019F460E820E00EC0A2E0FA1619F46EE30B
:1042A00024E108C0B3E0FB1619F466E12AE002C07D
:1042B00060E820E8812F90E030E0002341F08F7724
:1042C0009070821793075CF4212F2F5F38C08F778F
:1042D0009070281739071CF0212F215030C0462F2D
:1042E00050E0812F90E08F779070481759071CF0AD
:1042F000212F2E7F04C0212F261B2C7F260F211754
:1043000019F0002319F41BC0002361F0822F90E004
:104310008F7790708417950714F482E001C084E0D1
:10432000280F0DC0822F90E08F77907048175907A3
:1043300014F082E001C084E0281B01C0212F80918D
:10434000490283FF03C020934D02207820934B0243
:10435000F3C29091490297FF21C088E0892780939A
:10436000490283FF0EC080914B0280934D028078FA
:1043700080934B0210924C0286E699E160E971E06D
:104380000AC080914D0280934B0210924D0280E052
:1043900090E060E070E00E944C15CEC280914A022D
:1043A0008370813029F480E068E272E00E94E816B0
:1043B00080914B028058807880934B0210924C027F
:1043C00080914902877FAEC280912F029091300286
:1043D000009709F07DC0E0904502F0904602009100
:1043E0004702109148021E141F04100611060CF01B
:1043F0006FC0D0904A028D2D0E94EB1790E0A0E094
:10440000B0E08E159F05A007B1070CF458C081E0FD
:1044100090E0A0E0B0E00E2C04C0880F991FAA1F06
:10442000BB1F0A94D2F7209133023091340240919D
:1044300035025091360282279327A427B52780930F
:10444000330290933402A0933502B09336028091E8
:104450004902806880934902E0E1EE16F10401050B
:1044600011050CF4BAC160912D0270912E02C501A4
:104470000E949E26209133023091340240913502F1
:1044800050913602CA01AA27BB278F778B8377E129
:1044900056954795379527957A95D1F7822F8F773F
:1044A0008C8367E056954795379527956A95D1F7A0
:1044B0002D8380E06DE0A5010E94F4268EC1F3E01B
:1044C000DF22DF1609F038C28DE292E061E040C1E0
:1044D0006091490267FF10C0892B71F0809137020B
:1044E0009091380221E030E08227932790933802A0
:1044F00080933702606119C0809133029091340239
:10450000A0913502B091360221E030E040E050E069
:1045100082279327A427B5278093330290933402F0
:10452000A0933502B09336026F7E6093490204C2B5
:1045300080912F0290913002892B29F480914902B9
:104540008F77809349028091490285FFF5C1809160
:10455000450290914602A0914702B0914802181678
:1045600019061A061B060CF0F9C08DE292E060E015
:104570000E949F18F3C086E0FE013796DF011D926E
:104580008A95E9F78091450290914602A0914702F1
:10459000B09148020097A105B10509F454C0893FC4
:1045A000E7E09E07E0E0AE07E0E0BE070CF0C4C124
:1045B0008C0101501040000F111FC9018F779070BE
:1045C0000E9709F4016027FF23C01A8680914902E3
:1045D00083FD05C080E090E060E070E004C086E606
:1045E00099E160E971E00E944C1581E060E671E0BC
:1045F0000E94E81682E068E671E00E94E8161092D8
:10460000450210924602109247021092480202C0E0
:1046100081E08A87802F8F778F83C801880F892F49
:10462000881F990B91958F778887812F8295869522
:1046300086958370898780E066E0AE01495F5F4FB1
:104640000E94F42679C127FD77C1022F0D501091E9
:10465000490217FF0AC080912F0290913002892BE6
:1046600021F4213131050CF40C5F80914A020E9443
:10467000EB17081708F060C10430A0F08091F70331
:104680009091F803A091F903B091FA038C509E4FDA
:10469000AF4FBF4F80933D0290933E02A0933F02E5
:1046A000B093400217FF1DC080912F0290913002FD
:1046B000892BB9F082E090E0A0E0B0E004C0880F60
:1046C000991FAA1FBB1F0A95D2F72091370230917C
:1046D0003802282739273093380220933702106197
:1046E00020C082E090E0A0E0B0E004C0880F991FF5
:1046F000AA1FBB1F0A95D2F72091330230913402D2
:10470000409135025091360282279327A427B5277E
:104710008093330290933402A0933502B093360213
:104720001F7E1093490208C1809145029091460274
:10473000A0914702B09148020097A105B10509F484
:1047400084CF60E02F30310509F461E08DE292E022
:104750000E949F18809149028062E4C080914902C2
:104760008F7D8093490239C0809145029091460225
:10477000A0914702B09148020097A105B105B1F19F
:104780008091490282FD32C00E94740E833019F577
:1047900080914E02282F30E040E050E080914502A9
:1047A00090914602A0914702B0914802281739071C
:1047B0004A075B0744F42093450230934602409336
:1047C00047025093480280914B02807890914502B5
:1047D000892B80934B0210924C021092450210924A
:1047E00046021092470210924802A6C080E060E2A2
:1047F00043E00BC08091490287FF04C080E060E283
:1048000042E003C080E060E240E00E940A2794C0DA
:104810008091490287FF12C080913102909132024B
:10482000009709F48BC0A0E0B0E08093450290931C
:104830004602A0934702B09348021EC082FF21C0E7
:104840008091450290914602A0914702B0914802A2
:104850000097A105B105A9F486E00E9477458091F3
:10486000450290914602A0914702B09148020097FC
:10487000A105B10509F462C08DE292E00E94921F89
:104880005DC08091450290914602A0914702B0918F
:1048900048020097A105B10539F48FEF0E947745D2
:1048A00081E00E944A1B4AC079010027F7FC00956D
:1048B000102F6091450270914602809147029091BD
:1048C00048022AE030E040E050E00E94E44BE60E6F
:1048D000F71E081F191FF0E0EF16F0E8FF06F0E0E2
:1048E0000F07F0E01F0754F5E0924502F0924602F0
:1048F00000934702109348021FC08DE292E00E948D
:10490000921F1AC0809149028F770CC01092450205
:10491000109246021092470210924802809149027A
:104920008B7F80688093490207C080914B0280781A
:1049300080934B0210924C020E94770E2C960FB679
:10494000F894DEBF0FBECDBFCF91DF911F910F91C5
:10495000FF90EF90DF90BF90AF9008951F93182FB6
:10496000823118F02AEC37E032C00E943725FC0172
:104970002581243039F0253079F0812F90E02130E5
:10498000F1F414C0212F30E054E0220F331F5A9568
:10499000E1F7265B3C4F1BC0212F30E044E0220FA3
:1049A000331F4A95E1F726593B4F11C09C0194E013
:1049B000220F331F9A95E1F726573A4F08C09C0102
:1049C00084E0220F331F8A95E1F72655394FC9013C
:1049D0001F910895882319F02FE138E016C00E9436
:1049E0003725FC018581843029F0853031F0813014
:1049F00051F406C02BED37E008C02CEE37E005C0BF
:104A00002DEF37E002C02EE038E0C90108951F9372
:104A1000182F833218F02BE731E126C00E9437258A
:104A2000FC018581843029F0853051F08130B1F46A
:104A30000EC081E1189F90011124215D374F14C0F1
:104A400081E1189F900111242E57354F0DC081E14F
:104A5000189F900111242B52334F06C081E1189FFB
:104A600090011124285D304FC9011F9108958FE5F1
:104A700092E0089590915F02982309F091E0892FC8
:104A80000895ECEFFFEF25913591459154915070C9
:104A9000B901CA010895EFEFFFEF8491823029F444
:104AA000079902C080E8089582E00895FC01848D92
:104AB00081FD02C020E006C020E080819181892B29
:104AC00009F021E0822F0895FC01848D81FD02C050
:104AD00020E006C020E082819381892B09F021E04B
:104AE000822F0895F89488E181BD8BE081BDFFCFCE
:104AF000BF92CF92DF92EF92FF920F931F93CF93CB
:104B0000DF93082F6B01EA014115510529F10E943D
:104B1000F8177C0110E086E0B82E80E0602FA60137
:104B20000E94F426B0922A0402C00E947B0EC701A4
:104B3000FE010995882321F480912A048823A9F78E
:104B40000E94AA26811110E0C701FE010995882361
:104B500019F41F5F1A3008F3DF91CF911F910F9165
:104B6000FF90EF90DF90CF90BF900895DF93CF93A9
:104B700000D000D000D0CDB7DEB76115710531F19E
:104B80004115510519F1FE01319686E0DF011D92B4
:104B90008A95E9F7862F8F778983660F672F661FBF
:104BA000770B7195862F8F778A83842F8F778B83EE
:104BB000440F452F441F550B5195842F8F778C83BD
:104BC00082E0BF0144E655E20E94782526960FB6A2
:104BD000F894DEBF0FBECDBFCF91DF910895DF9374
:104BE000CF9300D000D000D0CDB7DEB761157105EE
:104BF000C1F0FE01319686E0DF011D928A95E9F74A
:104C0000862F8F778983660F672F661F770B7195C5
:104C1000862F8F778A8381E0BF0146E555E20E94A7
:104C2000782526960FB6F894DEBF0FBECDBFCF9184
:104C3000DF910895CF93DF93C0E0D0E0CE010E94D2
:104C4000684EFE01E15AFD4F6081861719F0CE01D2
:104C50000E94704EA8952196C032D10579F7DF9158
:104C6000CF910895809590915F02982390935F0271
:104C70000E941A26089590915F02982B90935F02EC
:104C80000E941A260895809364020E941A260895AD
:104C900090916402973008F091E080E1EFE5F2E056
:104CA000DF011D928A95E9F788E180936302909372
:104CB00064020E941A2608958FE592E060E070E099
:104CC00040E250E00E94584E809161029091620251
:104CD0008F5F9F4F11F40E944826809164028730B5
:104CE00010F010926402EAEFFFEF9491892F815047
:104CF0008E3F10F490936F000895FC0120E090E047
:104D000037E08191982780E097FF03C0990F9327A0
:104D100001C0990F8F5F8830B9F72F5F283089F76E
:104D200097FD9095892F089520917F023091800200
:104D30009093800280937F02C9010895FC01862F21
:104D40008F778083660F672F661F770B71956F775C
:104D50006183089580918902882319F01092890255
:104D600081E00895E0918102F0918202309709F08C
:104D7000099508958091020108950F931F93DF9381
:104D8000CF93CDB7DEB729970FB6F894DEBF0FBE2D
:104D9000CDBFDA0180910201806889836A83FE01B8
:104DA00033969E01275F3F4F109721F08D918F77AB
:104DB000808301C010823196E217F307A9F78E01B4
:104DC0000F5F1F4FC8010E947D268987C8010E947E
:104DD000E21029960FB6F894DEBF0FBECDBFCF917B
:104DE000DF911F910F9108950F931F93CF93DF933E
:104DF000082F162FEA0102C00E947B0E802F612F20
:104E0000AE010E94BD268823B9F3DF91CF911F9197
:104E10000F910895DF93CF9300D000D000D0CDB78D
:104E2000DEB7FE01319696E0DF011D929A95E9F713
:104E30004983AF010E94F42626960FB6F894DEBF90
:104E40000FBECDBFCF91DF910895FF920F931F93B7
:104E5000CF93DF93082FEB014115510519F42FEF84
:104E60003FEF4FC080917F0290918002509380026B
:104E700040937F0290938202809381021092850278
:104E80008EEF9FEF90938402809383023093880289
:104E90002093870210E094E0F92E002361F080E077
:104EA000602FAE010E94F42606C00E947B0E809106
:104EB0008602882311F0F0922A04909185029923AA
:104EC00021F480912A04882381F780918902882324
:104ED00019F01092890210E0992319F41F5F18301D
:104EE000E0F28091810290918202909380028093FF
:104EF0007F021092820210928102209183023091EF
:104F00008402C901DF91CF911F910F91FF90089505
:104F100020E030E00E9425270895DF92EF92FF9273
:104F20000F931F93DF93CF93CDB7DEB729970FB6BB
:104F3000F894DEBF0FBECDBF8E010F5F1F4F21ED76
:104F4000E22E28E2F22EDD24D3941AC0C8010E947A
:104F50007D2699858917A1F419C0D092890210C0C5
:104F600080917F0290918002892B21F4F09280023F
:104F7000E0927F02E0917F02F0918002C8010995E2
:104F8000C8010E940C11892B09F704C08A81863060
:104F900039F7E3CF29960FB6F894DEBF0FBECDBF29
:104FA000CF91DF911F910F91FF90EF90DF900895C7
:104FB0002F923F924F925F926F927F928F929F9229
:104FC000AF92BF92CF92DF92EF92FF920F931F9317
:104FD000DF93CF93CDB7DEB729970FB6F894DEBF36
:104FE0000FBECDBF0E9441259B01AC0110E8612E90
:104FF0001FE3712E812C912C622273228422952230
:10500000B7E09594879477946794BA95D1F7A12CDB
:10501000A0ECBA2EAFE1CA2ED12CA222B322C42218
:10502000D522FEE0D594C794B794A794FA95D1F70A
:10503000E12CF12CE0EE0E2F112DE222F3220423BD
:10504000152375E115950795F794E7947A95D1F7AF
:105050006FE7262E312C412C512C22223322442260
:1050600055222DC0A8958A81843049F5CE0101963C
:105070000E947D269985891711F541C08D8190E0A8
:10508000A0E0B0E0681679068A069B06C1F48C8120
:1050900090E0A0E0B0E0A816B906CA06DB0679F4F5
:1050A0008B8190E0A0E0B0E0E816F9060A071B0744
:1050B00031F489818F778093020181E007C0CE01AE
:1050C00001960E940C11892B69F680E029960FB693
:1050D000F894DEBF0FBECDBFCF91DF911F910F912E
:1050E000FF90EF90DF90CF90BF90AF909F908F9008
:1050F0007F906F905F904F903F902F9008958E819A
:1051000090E0A0E0B0E0281639064A065B06B9F642
:10511000B5CF0F931F93DF93CF93CDB7DEB729970A
:105120000FB6F894DEBF0FBECDBF209102012068FC
:10513000298323E02A83282F2F772B83880F892F19
:10514000881F990B91958F778C83862F8F778D830E
:10515000852F869586958E8367FF02C080648E8337
:10516000CA0103E0969587950A95E1F78F778F83BB
:10517000842F8295807788878E010F5F1F4FC8012B
:105180000E947D268987C8010E94021129960FB6C8
:10519000F894DEBF0FBECDBFCF91DF911F910F916D
:1051A0000895AF92BF92CF92DF92EF92FF920F934A
:1051B0001F93DF93CF9300D000D000D0CDB7DEB7E0
:1051C0006C010E94F8175C01FE01319686E0DF0158
:1051D0001D928A95E9F7F6016181862F90E0FC0126
:1051E0003397E332F10508F0A4C2EA5BFF4FEE0FFC
:1051F000FF1F0590F491E02D0994D60112968C9131
:105200000E94480FF601878184700E94103291C27B
:10521000D5010D911C91F601838190E09695982F10
:10522000882797958795228130E0822B932B08174A
:10523000190709F07EC20E94C41AC8010E94A12F5A
:1052400078C2D60113968C911397E82FF0E0F6956B
:10525000FE2FEE27F795E79512968C91129790E026
:10526000E82BF92B15968C911597382F330F330FA8
:1052700020E016968C911697482F50E04F7750708B
:1052800013E0440F551F1A95E1F717968C9190E0A3
:105290008077907074E0959587957A95E1F7482B23
:1052A000592B422B532B683041F4CF01BA010E9495
:1052B000EF188091290482602FC0809129048160B9
:1052C00080932904D60117968C9180FD05C08091AA
:1052D0002904826080932904D60114966C91149756
:1052E00015968C9186FD6068CF010E94EF1A0E948E
:1052F00009181FC2F601668170E07695762F662741
:1053000077956795858190E0682B792B84810E9441
:10531000071F80912904846080932904E8CFD60177
:1053200014964C91149750E015966C91159770E077
:105330007695762F66277795679516962C91169712
:10534000922F9295990F990F907C80E0682B792B82
:1053500013968C91139790E09695982F88279795A0
:10536000879512962C9130E0642B752B822B932B12
:105370000E940219809129048860CECFF6016281D3
:1053800013818581E82FF0E0D60116964C9116978F
:1053900017968C911797282F30E014960C91E6FD04
:1053A0000068FE2FEE27FF0FFF0F50E04F77507081
:1053B00083E0440F551F8A95E1F7C901807790700B
:1053C000B4E095958795BA95E1F7482B592B812F35
:1053D00090E09695982F88279795879570E04E2BAB
:1053E0005F2BE3E036952795EA95E1F72170862B50
:1053F000972B602F0E942A199CC1F50122A133A18D
:105400002115310569F0822F8F778983220F232F91
:10541000221F330B3195822F8F778A8318E00EC0BD
:10542000D5018C918F7789838D919C91880F892FDD
:10543000881F990B91958F778A8310E0F501848DF1
:1054400080FD10610E944125262F2F772B83A7E036
:105450009695879577956795AA95D1F7262F2F77FB
:105460002C83F7E09695879577956795FA95D1F710
:10547000262F2F772D83E7E096958795779567956B
:10548000EA95D1F76770612B6E838FEF6BE04CC1AB
:105490000E9441257B018C019B01AC012F7730706C
:1054A00040705070D60114968C9190E0A0E0B0E06E
:1054B000281739074A075B0709F071C1A80197014E
:1054C00020783F734070507067E056954795379548
:1054D00027956A95D1F7F601858190E0A0E0B0E0CC
:1054E000281739074A075B0709F059C1A801970136
:1054F0002070307C4F7150709EE0569547953795DF
:1055000027959A95D1F7868190E0A0E0B0E0281722
:1055100039074A075B0709F042C1278180E090E024
:10552000A0EEB0E0E822F9220A231B2385E11695BC
:105530000795F794E7948A95D1F7822F90E0A0E041
:10554000B0E087709070A070B070E816F9060A0796
:105550001B0709F024C18381682F70E07695762FB0
:10556000662777956795828190E0682B792B611586
:10557000710509F414C1269526952695122F20FF52
:105580000BC0A5014C5D5F4FCB0160E070E00E9455
:10559000492DBC01009721F0809102010E94EF2566
:1055A000D5018D919C911197892B09F4F8C011FFB9
:1055B000F6C05C968C915C9781605C968C93EFC092
:1055C000F601838190E09695982F88279795879587
:1055D000228130E0822B932B90932C0480932B0418
:1055E000A8C0D60113968C91139790E09695982FAA
:1055F00088279795879512962C91129730E0822BE9
:10560000932B90932F0480932E0414968C911497CF
:1056100080933C0415968C911597809330041696D0
:105620008C918093310480912D04816012C022E01E
:1056300030E0F601E20FF31F8081F901E05DFB4FDE
:1056400080832F5F3F4F2730310599F780912D04DC
:10565000826080932D046DC0F601828180933704AF
:105660008381809338048481809339048581809379
:105670003A0480912D048460ECCFD60115968C916C
:105680001597882309F455C013968C911397482FCA
:1056900050E05695542F44275795479514962C91D2
:1056A0001497922F9295990F990F907C80E0482B38
:1056B000592B12968C9190E0482B592B40FD02C03B
:1056C00067E601C062E7CA01969587950E94DC2FC4
:1056D00030C00E947225F60182810E94EA1829C01A
:1056E000D60112968C91882329F00E943725FC015F
:1056F000848101C080E00E9484151BC090E0D60127
:1057000012968C91811191E09093860212C0F6015D
:105710008281882371F48DE0898382E08A8381E02D
:105720008B838C838FEF6CE1AE014F5F5F4F0E94E4
:10573000F426D6012C9130E02F7730708091020151
:1057400090E02817390749F480912A04882329F02A
:1057500080912A04815080932A04F501848D81FD73
:1057600006C080E090E060E040E050E016C084FFBA
:105770000EC0D50112968D919C911397009739F028
:105780001A964D915C911B975E966C9106C0F5013F
:105790004681578180819181668D0E948928269655
:1057A0000FB6F894DEBF0FBECDBFCF91DF911F9132
:1057B0000F91FF90EF90DF90CF90BF90AF90089542
:1057C0009093840280938302209187023091880213
:1057D0002115310549F06115710531F0411551056B
:1057E00019F0C9010E942C4C81E080938502089534
:1057F00060E070E040E050E00E94E02B0895DF930D
:10580000CF9300D000D000D0CDB7DEB7FE013196E7
:1058100026E0DF011D922A95E9F7282F2F772983AB
:10582000880F892F881F990B91958F778A838FEF27
:1058300063E1AF010E94F42626960FB6F894DEBF0E
:105840000FBECDBFCF91DF910895DF92EF92FF920F
:105850000F931F93DF93CF9300D000D000D0CDB72C
:10586000DEB7E62EFE01319626E0DF011D922A9575
:10587000E9F7282F2F772983880F892F881F990B05
:1058800091958F778A838FEF9FEF90932C0480936D
:105890002B0410E0FE2E0F2F35E0D32E16C08FEF15
:1058A0006E2D4F2D502F0E94F426D0922A0402C054
:1058B0000E947B0E80912B0490912C0497FF04C0D2
:1058C00080912A048823A1F71F5F80912B04909177
:1058D0002C0497FF02C01A3011F720912B0430914D
:1058E0002C04C90126960FB6F894DEBF0FBECDBFBB
:1058F000CF91DF911F910F91FF90EF90DF9008956E
:1059000062E10E94252C089561E10E94252C0895F2
:105910008F929F92AF92BF92CF92DF92EF92FF92BF
:105920000F931F93DF93CF9300D000D000D0CDB75B
:10593000DEB7FC0179016115710509F48AC02115F2
:10594000310509F486C06E010894C11CD11C86E0A3
:10595000D6011D928A95E9F7CB01880F892F881F00
:10596000990B9195BFE79B2E982214E1AFE7AA2EE1
:10597000A6227FE7B72EB42265E0862E8E2F8F7782
:105980008983EE0FEF2FEE1FFF0BF1958E2F8F7790
:105990008A83163171F0173128F4143171F0153102
:1059A00031F505C0173139F0183109F50AC090E01A
:1059B0000CC080E008C080E005C0AB829C82BD8244
:1059C00016C083E08D5F982F9D5FF701E90FF11DF1
:1059D00080818B83892F8F5FF701E80FF11D908104
:1059E0009C838F5FF701E80FF11D80818D831092FA
:1059F0002C0410922B0400E015C08FEF612FA6013C
:105A00000E94F42680922A0402C00E947B0E80919C
:105A10002B0490912C04892B21F480912A04882353
:105A2000A1F70F5F80912B0490912C04892B11F426
:105A30000A3019F780912B0490912C04892B49F09E
:105A4000E0912B04F0912C041F5F193109F096CFDF
:105A500002C0E0E0F0E0CF0126960FB6F894DEBF7A
:105A60000FBECDBFCF91DF911F910F91FF90EF90AF
:105A7000DF90CF90BF90AF909F908F900895FC01E2
:105A8000A62F9A0180E090E0BF014A2F0E94882C47
:105A90000895AF92BF92CF92DF92EF92FF920F9351
:105AA0001F93DF93CF9300D000D000D0CDB7DEB7E7
:105AB0009C018B017A0101978F5F934008F06CC0C5
:105AC000FE01319686E0DF011D928A95E9F7822F6B
:105AD0008F778983220F232F221F330B3195822F3B
:105AE0008F778A8310922D04DD24BE2ECF2E8FE077
:105AF000A82E1EC08FEF60E14B2D5C2D0E94F42676
:105B0000A0922A0402C00E947B0E80912D0487304F
:105B100021F080912A048823B1F780912D048730E9
:105B200031F082B790E08C599F4F0E948E12D3942F
:105B300080912D04873019F0BAE0DB16D9F68091F8
:105B40002D04873021F4809130048F3759F40115EA
:105B5000110511F0F8011082E114F104E9F0D70108
:105B60001C921AC00115110521F080913C04F80126
:105B70008083E114F10459F0D701E0E3F4E08BE015
:105B800001900D928150E1F7D7011B961C92209154
:105B90002E0430912F0402C020E030E0C901269687
:105BA0000FB6F894DEBF0FBECDBFCF91DF911F912E
:105BB0000F91FF90EF90DF90CF90BF90AF9008953E
:105BC00010923E0490913E0490933D0490913D04C8
:105BD000909360049091600490935F04119A1098E0
:105BE000199A189892E09BB9883008F087E0E82F5E
:105BF000F0E0EE0FFF1FE857FE4EA591B49165301F
:105C000010F465E003C0693008F068E04F7D65502E
:105C1000660F453411F4606203C04F3409F46063C9
:105C2000223008F068608B2F992787FD9A958F7036
:105C300080939000A9B96093950088EB8AB980E0C1
:105C400090E008951F920F920FB60F9211248F9338
:105C50009F93EF93FF9390915F0480916004981756
:105C600011F4559812C0E0916004F0E0E35CFB4F42
:105C700084A18CB9809160048F5F809360048091CF
:105C80006004803210F010926004FF91EF919F91B8
:105C90008F910F900FBE0F901F9018951F920F922B
:105CA0000FB60F9211242F933F938F939F93EF93EF
:105CB000FF9320913D0480913E0430E090E00197F5
:105CC0002817390741F080913D048F3179F4809194
:105CD0003E04882359F480913E048F5F80933E04F4
:105CE00080913E04803210F010923E04E0913D0419
:105CF000F0E08CB1E35CFB4F828380913D048F5FC9
:105D000080933D0480913D04803210F010923D0458
:105D1000FF91EF919F918F913F912F910F900FBE27
:105D20000F901F90189527E0813D9207C0F12FE05A
:105D3000813A920710F481E01EC023E28932920773
:105D400010F482E018C026E3813B920710F483E050
:105D500012C026E48135920710F484E00CC028E8D4
:105D6000893B920710F485E006C0895D964D10F0DE
:105D700087E001C086E0789420E030E05E9902C0C0
:105D800020E030E02F5F3F4FA89597E220313907A0
:105D9000A8F368E04EE421E00E94E02D089580E041
:105DA000EACF8330C9F0843028F4813061F082304A
:105DB00080F40CC08530B1F0853088F08630A9F0D1
:105DC0008730C9F415C020E639E017C020EB34E075
:105DD00014C020EC32E111C020E835E20EC020E40E
:105DE00038E30BC020E03BE408C020E036E905C002
:105DF00020E031EE02C020E030E0C901089539B161
:105E000020919000922F80E0232F30E0282B392B17
:105E100048E851E160E0FA01859194918217930777
:105E200029F06F5F4E5F5F4F6830A9F7862F0E94A1
:105E3000D12E0895482FA89503C0559A7894A89517
:105E400020915F048091600430E090E00197281772
:105E5000390799F380915F048F3121F480916004B8
:105E6000882359F3E0915F04F0E0E35CFB4F44A327
:105E70009FB7F89480915F048F5F80935F04809157
:105E80005F04803210F010925F049FBF559A80E04B
:105E900090E0089590913D0480913E04981719F484
:105EA0002FEF3FEF15C0E0913E04F0E0E35CFB4FC5
:105EB0009281F89480913E048F5F80933E0480919C
:105EC0003E04803210F010923E04292F30E0789486
:105ED000C9010895CF92DF92EF92FF920F931F9323
:105EE000CF93DF93E82E162F042FF52E6AEC0E9435
:105EF000FC168E2D612F0E94FC16802F9F2DEC0129
:105F000085E0C82ED12CCC0EDD1E0FC01881812F4C
:105F10008A5C843028F48E2D6BEC0E94FC161F7076
:105F20008E2D612F0E94FC162196CC15DD0571F790
:105F3000DF91CF911F910F91FF90EF90DF90CF9065
:105F40000895DF93CF9300D000D000D0CDB7DEB757
:105F5000FE01319626E0DF011D922A95E9F799832B
:105F60008A8380E063E0AF010E946A2F26960FB615
:105F7000F894DEBF0FBECDBFCF91DF910895DF93C0
:105F8000CF9300D000D000D0CDB7DEB7FE01319660
:105F900096E0DF011D929A95E9F7898380E062E03F
:105FA000AF010E946A2F26960FB6F894DEBF0FBE8F
:105FB000CDBFCF91DF910895DF93CF9300D000D074
:105FC00000D0CDB7DEB7FE01319626E0DF011D928D
:105FD0002A95E9F799838A836F776B8380E066E07F
:105FE000AF010E946A2F26960FB6F894DEBF0FBE4F
:105FF000CDBFCF91DF910895EF92FF920F931F9342
:10600000DF93CF93CDB7DEB762970FB6F894DEBFBC
:106010000FBECDBF162F882309F094C18091940242
:106020008823B1F060918A0270918B0280918C027A
:1060300090918D026C5E7F4F8F4F9F4F0E94E311B6
:10604000882331F0109294021092950210929602D9
:106050008091F7039091F803A091F903B091FA03AE
:1060600080938A0290938B02A0938C02B0938D024E
:106070001A3C41F4109294021092950281E08093B0
:10608000960260C180919602882309F45BC11B3C93
:1060900021F481E08093950255C180919502811190
:1060A000106C1092950280919402E82FF0E0E65770
:1060B000FD4F14838F5F80939402863008F442C1B1
:1060C0000E94F8178C0190918E02933009F4B4C0AD
:1060D000943030F4913059F1923008F055C00AC034
:1060E000953009F4C5C0953008F4B4C0963009F075
:1060F0001FC1E8C080E06CEC0E94FC16D801169627
:106100008D919C9117979C012E7F3F77369527950F
:1061100080FD3068F801868D8F83388729870E943B
:10612000740E8A871C861B8680E060E027C080E0B2
:106130006CEC0E94FC16D80111968C9111978F83FC
:106140005C915D964C915D97242F30E02370307008
:1061500094968C91992787FD9095282B392B232B8A
:1061600011F480E001C080E858878987842F0E945D
:10617000E1178A871C861B8680E061E0AE01495FDB
:106180005F4F0E946A2FD8C090918F0280E02091CB
:106190009002BC01620F711D9091920280E02091EB
:1061A0009302820F911DAC01440F551F4E7F5F7704
:1061B00097FD41606115710519F4F80160817181E5
:1061C000F0E460307F0708F0B3C0D8018D919C9156
:1061D0006817790739F4CB016091910220E00E94A1
:1061E0002A196DC0862F8F778983660F672F661FE8
:1061F000770B7195862F8F778A8390919102892FE3
:106200008F778B83852F869586958C8397FF02C029
:1062100080648C83CA0133E0969587953A95E1F7BF
:106220008F778D83842F829580778E8380E063E0E3
:10623000AE014F5F5F4F41C090918F0280E020918F
:106240009002820F911D60E00E94281F882309F4AC
:106250006FC035C040918F02442329F0842F8250B3
:10626000823008F065C080E060E20E940A2727C003
:1062700030918F0220E080919002280F311DFE01A5
:10628000319686E0DF011D928A95E9F7822F8F779C
:106290008983C901880F892F881F990B91958F7762
:1062A0008A83832F82958695869583708B838091D0
:1062B00091028C8380E066E0AF010E94F42680E0CA
:1062C0006CEC38C030918F0220E080919002280F52
:1062D000311D8E01035F1F4FF80111929A95E9F766
:1062E000F22EE32EC801B9010E949E2689E1B80171
:1062F0004FEA51E30E9488278C018235910569F0AD
:106300008335910524F48734910591F406C08736CE
:10631000910519F08237910559F480E06CEC0E94E8
:10632000FC16602F6F778F2D9E2D0E94DC2F04C0EE
:1063300080E06DEC0E94FC1610929402109295027F
:106340001092960262960FB6F894DEBF0FBECDBFD4
:10635000CF91DF911F910F91FF90EF900895FC0175
:106360008181893121F0CF010E94B2260895848174
:1063700090E00E94F82B0895FB0157FD02C021E038
:1063800004C0509541955F4F20E08330910541F165
:106390008430910534F48130910501F1029751F573
:1063A00023C08430910519F0059721F50AC0818139
:1063B0008F5F818390E084179507E4F0222351F0EA
:1063C0000DC081818150818390E08417950794F0FE
:1063D000222321F0842F815081830CC011820AC0B6
:1063E00012821382168A06C090E08281882309F403
:1063F00091E0928380E090E008958230910519F059
:10640000039751F403C02FEF3FEF08C083E090E003
:1064100040E050E00E94BC3120E030E0C901089526
:106420001F93182F0E94F817FC01848D112311F07F
:10643000806401C08F7B848F1F9108951F93CF9339
:10644000DF93EC018A81882309F470C081E060E069
:106450000E94071600D000D00F92EDB7FEB731961C
:1064600012E0ADB7BEB711961C9384E092E192831F
:1064700081838C819D81948383830E9475170F9003
:106480000F900F900F900F908B81843079F400D093
:106490000F92EDB7FEB7118380E092E19383828380
:1064A0000E9475170F900F900F9018C000D000D069
:1064B0000F92EDB7FEB73196ADB7BEB711961C93EC
:1064C0008CEF91E1928381838885838314820E947B
:1064D00075170F900F900F900F900F90898D9A8DD8
:1064E00097FD04C082E064EF71E10CC08E5F9F4FA6
:1064F00021F482E06CEE71E105C084E00E94072582
:10650000BC0182E00E94CF1781E0888F8E8B8B8147
:10651000813058F0833020F08450823030F402C053
:1065200083E001C088E08F8B01C01E8ADF91CF918C
:106530001F9108959C01FB018130910569F0823023
:1065400091051CF40097D9F027C083309105F1F034
:106550008530910509F517C08EEF9FEF928F818FDF
:106560004091A6025091A702CA0101978050944021
:1065700018F45583448310C0358324830DC0CB01A8
:106580000E941E3209C081E0838306C083E090E050
:1065900040E050E00E94BC3180E090E008951F93FD
:1065A000182F81E060E00E940716113049F0113089
:1065B00028F0123039F0133071F406C083E105C0C1
:1065C00084E103C085E101C086E10E940725BC018A
:1065D00082E00E94CF171F9108951F93CF93DF93FE
:1065E000EB018230910509F493C0833091051CF4CE
:1065F000892B31F0BBC0863091050CF0B7C075C057
:1066000081E060E00E9407168A818823A1F000D013
:1066100000D00F92EDB7FEB7319682E0ADB7BEB7AE
:1066200011968C9386EB91E1928381838C819D817D
:106630009483838346C020919702309198024091C1
:10664000990250919A02211531054105510509F42D
:1066500040C08DB79EB707970FB6F8949EBF0FBE88
:106660008DBFEDB7FEB7319612E0ADB7BEB711964C
:106670001C938EEA91E19283818323833483458343
:1066800056830E9475176C817D818DB79EB70796E2
:106690000FB6F8949EBF0FBE8DBF6115710509F44A
:1066A00065C000D000D00F92EDB7FEB73196ADB700
:1066B000BEB711961C9389EA91E19283818374831A
:1066C00063830E9475170F900F900F900F900F909B
:1066D0004DC08C819D8197FF49C084E00E940725B1
:1066E000BC0182E00E94CF1741C08330910551F474
:1066F00010929702109298021092990210929A02A8
:106700001D821C82BE0142E050E00E94BC312EC0BE
:106710008A81882371F41D821C8283E08B838FEF32
:106720009FE39F838E8391E0988F85E08F8B9E8B74
:1067300017C01E8A8C819D810E943C4A60939702FB
:10674000709398028093990290939A021B8261152C
:1067500071058105910521F48FEF9FEF9D838C8357
:1067600090E08A81882309F491E09A8380E090E0A8
:10677000DF91CF911F910895FF920F931F93CF93B5
:10678000DF93EC018B01F42E0E943725FC01C2300F
:10679000D10509F48BC0C330D10534F42097D1F072
:1067A000219709F09BC00DC0C430D10509F463C026
:1067B000C430D1050CF463C0C530D10509F08EC0DA
:1067C0005EC0FF2019F08485D8016DC08385F80173
:1067D000818384C081E060E00E940716FF2059F1A8
:1067E000D80111962C91EDB7FEB737970FB6F894F4
:1067F000FEBF0FBEEDBF319682E0ADB7BEB71196BA
:106800008C9381EC91E192838183822F6AE00E94D4
:10681000034C83831482822F0E94034C958316823B
:106820000E947517EDB7FEB737960FB6F894FEBF06
:106830000FBEEDBF53C000D000D00F92EDB7FEB732
:10684000319682E0ADB7BEB711968C938BEB91E198
:1068500092838183D80111968C9122E3829FC0019B
:106860001124948383830E9475170F900F900F90CB
:106870000F900F9033C0F80181818F3F79F1FF2095
:1068800019F44BEE5FEF02C040E05FEFCE01B801BC
:106890000E94BC31FF2011F1D80111968C91119703
:1068A0008823E1F481E011968C9318C0D8011296E8
:1068B0008C911297882349F011968C91FF2011F04A
:1068C000848701C083870E941A2690E0F8018281A4
:1068D000882309F491E0D80112969C9380E090E01F
:1068E000DF91CF911F910F91FF90089541E00E9499
:1068F000BC33089540E00E94BC3308951F93CF93AA
:10690000DF93EB0182309105C1F18330910534F4BE
:106910000097C1F0019709F04CC005C08630910581
:106920000CF047C025C00E943725FC01808185FFFF
:1069300002C082E003C084FF03C081E0898339C0C4
:10694000198237C081E060E00E9407168981825F6A
:106950000E94072500D00F9222E0EDB7FEB72183F9
:10696000938382830E9475170F900F900F9021C020
:1069700043E050E00E94BC311CC08A81882399F01A
:106980000E943725FC0110811F7C8981813011F420
:10699000106103C0823009F410620E943725FC01A7
:1069A00010830E941A2690E08A81882309F491E0DE
:1069B0009A8380E090E0DF91CF911F910895CF936B
:1069C000DF93EB018230910581F1833091052CF446
:1069D000009781F00197C9F504C086309105ACF5A8
:1069E0001FC00E943725FC0187818983843068F1AC
:1069F00019822BC081E060E00E9407168981865FC2
:106A00000E94072500D00F9222E0EDB7FEB7218348
:106A1000938382830E9475170F900F900F9015C07B
:106A200044E050E00E94BC3110C08A81882339F0D4
:106A30000E9437252981FC0127830E941A2690E0B5
:106A40008A81882309F491E09A8380E090E0DF91C5
:106A5000CF9108951F93CF93DF939C01EB01823078
:106A6000910509F484C0833091053CF4009749F105
:106A70008130910509F0AEC005C0863091050CF05B
:106A8000A9C070C08C819D8101978C5F934010F0EC
:106A90003D832C838CEF93E09F838E8311E01B83D7
:106AA0001E8B83E08F8B188F8C819D810197880FBF
:106AB000991F0E942D481982039709F08BC01983F2
:106AC00089C081E060E00E9407168B81813079F5F2
:106AD0002C813D818DB79EB707970FB6F8949EBF66
:106AE0000FBE8DBFEDB7FEB7319682E0ADB7BEB732
:106AF00011968C9383E091E0928381833483238386
:106B00002D5F3F4F368325830E94A2178DB79EB716
:106B100007960FB6F8949EBF0FBE8DBF89818C5F1C
:106B20000E94AE24BC0182E00E94CF1753C000D067
:106B300000D00F92EDB7FEB7319682E0ADB7BEB789
:106B400011968C938DE091E0928381838C819D815D
:106B5000948383830E94A2170F900F900F900F9041
:106B60000F9038C042E050E00E94BC3133C08A81AF
:106B7000882399F02C813D818981882319F461E073
:106B800070E002C063E070E021503040C901880F1E
:106B9000991F0E9402481A821DC08B81813019F40E
:106BA0008A831E8A17C08C819D8101978C7F0196F4
:106BB0009D838C830197880F991F0E942D4819820D
:106BC000039711F481E0898391E09B839E8B83E09E
:106BD0008F8B988F80E090E0DF91CF911F91089587
:106BE000CF93DF93EB018230910541F18330910522
:106BF0002CF4009789F00197E9F504C086309105DF
:106C0000CCF517C080E090E00E942D4819820397D0
:106C100089F581E089832EC081E060E00E9407163B
:106C200089818E5F0E94AE24BC0182E00E94CF1752
:106C300021C042E050E00E94BC311CC08A81882300
:106C400099F081E060E00E94071682E069EC71E152
:106C50000E94CF178981882319F481E090E002C057
:106C600083E090E00E94DE4790E08A81882309F467
:106C700091E09A8380E090E0DF91CF910895CF93E7
:106C8000DF93EB018230910509F450C08330910508
:106C900034F4009769F0019709F054C005C08630BC
:106CA00091050CF04FC03DC00E942B4989834AC01A
:106CB00081E060E00E94071669816623A9F48CE1F7
:106CC0000E94072500D00F9222E0ADB7BEB7119603
:106CD0002C93119713969C938E9312970E9475177D
:106CE0000F900F900F902EC000D000D00F92EDB7F4
:106CF000FEB7319682E0ADB7BEB711968C9388EDA2
:106D000091E19283818385E0689FC001112494837F
:106D100083830E9475170F900F900F900F900F9024
:106D200011C049EC50E00E94BC310CC08A8188231C
:106D300019F089810E94034990E08A81882309F42F
:106D400091E09A8380E090E0DF91CF9108951F93C6
:106D5000CF93DF93EB01122F8230910519F183302D
:106D600091052CF4009761F0019779F504C0863005
:106D700091055CF512C0842F0E94144B898325C0B5
:106D800081E060E00E9407168981810F0E94AE2495
:106D9000BC0182E00E94CF1718C042E050E00E9480
:106DA000BC3113C08A81882351F08981882321F066
:106DB000842F0E94744B03C0842F0E94484B90E0A4
:106DC0008A81882309F491E09A8380E090E0DF9142
:106DD000CF911F91089544E026E00E94A7360895C0
:106DE00041E020E00E94A736089548E022E00E949A
:106DF000A7360895CF93DF93EB018130910569F0B9
:106E0000823091051CF4892B69F04CC082309105C9
:106E100079F1039709F046C024C00E94E2489D839F
:106E20008C8340C081E060E00E94071600D000D053
:106E30000F92EDB7FEB7319682E0ADB7BEB71196AF
:106E40008C938EED91E1928381838C819D819483DB
:106E500083830E9475170F900F900F900F900F90E3
:106E600021C083E090E040E050E00E94BC311AC0B5
:106E70008A81882361F483E08B8384E390E09F839D
:106E80008E8391E0988F82E08F8B9E8B05C01E8A47
:106E90008C819D810E94C14890E08A81882309F4F9
:106EA00091E09A8380E090E0DF91CF910895CF93B5
:106EB000DF93EB018230910581F18330910534F449
:106EC0000097C9F0019709F044C005C086309105CC
:106ED0000CF03FC01DC00E943D46813051F0813012
:106EE00018F0833029F402C0198233C082E001C057
:106EF00083E089832EC081E060E00E9407168981CB
:106F0000885F0E94AE24BC0182E00E94CF1721C09E
:106F100044E050E00E94BC311CC08A81882399F073
:106F20008981813049F0813028F0823039F0833016
:106F300051F406C080E005C081E003C083E001C0D9
:106F400087E00E94034690E08A81882309F491E05B
:106F50009A8380E090E0DF91CF910895CF93DF9303
:106F6000EB018230910549F1833091051CF4892BA6
:106F700029F02EC0863091055CF51AC08A818823DD
:106F800039F180E061E00E94071681E20E94072546
:106F9000BC0182E00E94CF1781E060E00E940716EA
:106FA00089E10E940725BC0182E00E94CF1710C032
:106FB00040E050E00E94BC310BC08A81882311F070
:106FC0000E944B4990E08A81882309F491E09A83DA
:106FD00080E090E0DF91CF9108950F931F93CF93BE
:106FE000DF93FC018B01EA0180819181892B21F0E3
:106FF000858D8370833081F081E060E00E94071608
:1070000085E00E940725BC0182E00E94CF1780E046
:107010000330110541F526C00E94740E833011F132
:107020000E94740E8230F1F00630110559F480E0B0
:1070300060E243E00E940A2781E090E0BE010E94E6
:107040009A320EC081E060E00E94071686E00E943E
:107050000725BC0182E00E94CF171A821B821E8A7C
:1070600080E001C081E0DF91CF911F910F910895E1
:10707000EF92FF920F931F93CF93DF938C01EB015D
:107080000E94F8177C01B801AE010E94ED378823F9
:1070900009F4B1C00230110509F491C003301105A3
:1070A00044F40115110549F10130110509F0A3C09F
:1070B0000DC00430110509F45EC0043011050CF454
:1070C00076C00530110509F096C062C08EEF9FEFC3
:1070D0009A8F898F2091A6023091A702C90101974A
:1070E0008050944018F43D832C8302C01D830C8390
:1070F00080E094E09F838E837EC08A81882309F498
:107100007AC081E060E00E9407162C813D8137FF44
:1071100014C000D00F9282E0ADB7BEB711968C9329
:10712000119787EE91E113969C938E9312970E948C
:1071300075170F900F900F9018C000D000D00F92CD
:10714000EDB7FEB7319682E0ADB7BEB711968C931E
:1071500083EE91E192838183348323830E947517A8
:107160000F900F900F900F900F9083E08F8B81E026
:10717000888F8E8B40C08C819D8101969D838C83EE
:107180002E813F81821793077CF03D832C830CC0B6
:107190008C819D8101979D838C831816190624F09C
:1071A00081E090E09D838C8381E08B8324C083E029
:1071B00090E0BE0140E050E00E94BC311CC091E074
:1071C0009B838A818823B1F02C813D81121613069E
:1071D00094F421503040F7018081918160E041E0DA
:1071E00000E00E945B468C819D819093A702809372
:1071F000A60201C09A8380E090E0DF91CF911F91B9
:107200000F91FF90EF9008950F931F93CF93DF930B
:10721000EC01062F142F8A818823F9F481E08B83F7
:10722000643019F488E090E002C080E094E09F832D
:107230008E832C813D818E819F818217930724F458
:1072400081E090E09D838C8381E08A83083009F49B
:10725000E0C080E00E94480FDCC08C819D8190934B
:10726000A7028093A602643009F1653060F46130B2
:1072700009F49EC06130D0F0623009F49BC06330E5
:1072800009F0C7C0C4C0673009F492C0683038F450
:10729000653009F48DC0663009F0BBC007C06830A6
:1072A00009F467C0693009F0B4C082C08B81815095
:1072B000823080F58EEF9FEF9A8F898FCE010E94EA
:1072C0001E3281E06AE00E94071681E10E940725D4
:1072D000BC0182E00E94CF17043051F0063069F003
:1072E000002391F48C819D8101970E9433470AC04D
:1072F0008C8181500E94604705C08C819D810197DF
:107300000E942E479A8F898F898D9A8D97FD56C03E
:10731000888754C081E06AE00E94071682E10E94DB
:107320000725BC0182E00E94CF17043061F00630CF
:10733000B9F0002309F042C08C819D8101976885D6
:107340000E94FF4613C08C819D81893091051CF0FD
:107350008FEF9FEF0BC0815068850E94384706C0B1
:107360008C819D81019768850E94F8469A8F898F4C
:1073700025C00E94F817FC0140815181411551053B
:10738000E9F0858D83708330C9F42C813D8121150E
:107390003105A1F08B818150823080F02150304046
:1073A000CA01612F40E008850E945B461B8231C004
:1073B00084E02EC08B818150823010F481E028C09F
:1073C00081E06AE00E9407168B81863071F481E1CA
:1073D0000E940725BC0182E00E94CF178C819D810D
:1073E000019769850E94B3470EC082E10E9407257C
:1073F000BC0182E00E94CF178C819D810197698535
:10740000498D0E9481479A8F898F86E001C087E06D
:107410008B83DF91CF911F910F9108950F931F934D
:10742000CF93DF93EC018B010E94F817BE01A801F6
:107430000E94ED378823F1F0C230D10549F0C43005
:10744000D105A1F4C80169E040E00E94043912C0EE
:10745000C80168E040E00E940439F8018381882374
:1074600049F40E9403162FEF3FEF06C0CE01B8018A
:107470000E949A3220E030E0C901DF91CF911F9144
:107480000F9108958230910531F08430910549F4CF
:10749000CB0167E002C0CB0166E040E00E94043906
:1074A00002C00E949A3280E090E0089582309105F7
:1074B00031F08430910549F4CB0165E002C0CB0185
:1074C00064E040E00E94043902C00E949A3280E0E9
:1074D00090E008958230910531F08430910549F4AF
:1074E000CB0161E002C0CB0160E040E00E940439C2
:1074F00002C00E949A3280E090E008951F93182FF6
:107500001816B4F480E00E94CF3280E090E0612F42
:107510000E94FF46892B39F48CE190E065E040E061
:107520000E94814707C0812F0E94A346892B11F03A
:1075300082E001C083E00E94CF3284EF91E00E949C
:107540008E121F910895CF92DF92EF92FF920F93C8
:107550001F93CF93DF937B018130910571F08230CF
:1075600091051CF4892B89F0D0C08230910509F473
:1075700052C0039709F0C9C047C08FEF9FEFDB01EE
:1075800015969C938E931497C0C0FB01828188232B
:1075900009F4BBC081E060E00E940716D701149691
:1075A0002D913C91159737FF10C000D00F9282E0CB
:1075B000EDB7FEB781838EE092E1938382830E94D0
:1075C00075170F900F900F9018C000D000D00F9239
:1075D000EDB7FEB7319682E0ADB7BEB711968C938A
:1075E0008AE092E192838183348323830E9475171A
:1075F0000F900F900F900F900F9085E0F701878B01
:1076000081E0808F868B81C083E090E040E050E095
:107610000E94BC317AC0DB0112968C9112978823AC
:1076200099F11496CD91DC911597C038D10520F4CD
:107630008C2F0E947E3A2FC0B0E4C030DB0708F0E8
:107640006FC080E00E94CF326E016D2D606C80E1D2
:1076500090E00E94FF46892B09F062C081E190E032
:107660006C2F0E94FF46892B09F05AC08CE190E0F4
:1076700065E041E00E94814783E00E94CF3284EFC1
:1076800091E00E948E1207C081E00E94CF3281E01B
:10769000D70112968C93F7018481958101978F37DA
:1076A000910550F480E090E00E943347D701159691
:1076B0009C938E93149715C080E190E00E9433470D
:1076C000182F00E0F7011583048381E190E00E9408
:1076D0003347082B192B1F73D70115961C930E9354
:1076E0001497F70184819581805098423CF08FEF88
:1076F0009FEFD70115969C938E93149781E0F70125
:1077000083838FEF97E29783868380E090E0DF9119
:10771000CF911F910F91FF90EF90DF90CF90089540
:1077200082E0ABCFCF93DF93EB018230910509F478
:107730004CC08330910509F441C0892B09F05DC02C
:107740008A81882309F459C081E060E00E9407160D
:107750002C813D8137FF14C000D00F9282E0ADB77D
:10776000BEB711968C93119789E192E113969C9381
:107770008E9312970E9475170F900F900F9018C05C
:1077800000D000D00F92EDB7FEB7319682E0ADB7D2
:10779000BEB711968C9385E192E192838183348305
:1077A00023830E9475170F900F900F900F900F90EA
:1077B00083E08F8B81E0888F8E8B1FC083E090E009
:1077C00040E050E00E94BC3118C08A81882321F03B
:1077D0008C810E947E3A05C081E00E94CF3281E018
:1077E0008A8380E090E00E9433479D838C8381E010
:1077F0008B838FE790E09F838E8380E090E0DF9122
:10780000CF910895CF93DF93EB018230910509F476
:107810008FC08330910534F40097B1F0019709F0DF
:107820008CC00CC08430910509F46DC08430910582
:107830000CF477C0059709F080C06BC081E090E040
:107840000E949A32198679C08A81882309F475C00A
:1078500081E060E00E9407168B81882331F482E08A
:107860006DE272E10E94CF1725C08DB79EB70797D2
:107870000FB6F8949EBF0FBE8DBFEDB7FEB7319621
:1078800082E0ADB7BEB711968C938EE192E1928300
:1078900081838C819D8194838383898585831682EE
:1078A0000E9475178DB79EB707960FB6F8949EBFC6
:1078B0000FBE8DBF898D9A8D97FD0AC082309105CC
:1078C0001CF0029729F402C0805D03C08FE301C061
:1078D00085E40E94C41581E0888F8E8B8B81863071
:1078E00059F0873020F48150823058F403C087303B
:1078F00041F404C086E003C08CE001C08EE08F8BB1
:107900001CC01E8A1AC08B81863041F4CB0163E013
:1079100011C08B81863011F481E001C086E08B8339
:107920000CC083E090E040E050E00E94BC3105C014
:10793000CB0162E040E00E94043980E090E0DF91FA
:10794000CF910895AF92BF92CF92DF92EF92FF92C4
:107950000F931F93CF93DF938C01EB01823091053E
:1079600009F491C0833091053CF4009771F08130A7
:10797000910509F0A1C05DC08330910509F455C09F
:10798000863091050CF098C06CC08A81882309F478
:1079900093C080919B02882309F48EC081E060E04F
:1079A0000E94071600D000D00F92EDB7FEB73196B7
:1079B00082E0ADB7BEB711968C9382E093E19283DB
:1079C00081838C819D81948383830E9475170F909E
:1079D0000F900F900F900F9089810E94A0485C013A
:1079E000C12CE0E8DE2E70E8E72EF12C00E010E07C
:1079F000C6018A219B21892B11F424E001C026E0D5
:107A0000C7018A219B21892B09F02F5F822F0E94B9
:107A1000C415F694E7940F5F1F4F0830110519F055
:107A2000D694C794E5CF1E8A47C01E8A81E00E9483
:107A300058480E94E24880939B0284E068E072E02C
:107A40000E94E81685E060E172E00E94E81686E098
:107A500068E172E00E94E81687E060E272E00E944E
:107A6000E81640919B02C801BE0150E00E94BC3163
:107A7000898190E001969D838C838B818230E1F433
:107A800088E08B8319C08A81882389F481E090E0A3
:107A90009D838C8380919B028E831F8211E01A83C9
:107AA00080E00E945848188F85E08F8B1E8B88E0FD
:107AB0008B838C818150898380E090E0DF91CF912E
:107AC0001F910F91FF90EF90DF90CF90BF90AF90FC
:107AD00008951F9380919D02803178F010929D024D
:107AE00010929C0281E061E00E94071610E085EA96
:107AF0000E94C4151F5F1F30D1F781E060919D0285
:107B00000E94071680919C02813039F0813018F074
:107B1000823091F406C085E001C084E00E94C41563
:107B20000BC080E20E94C41585E00E94C4158091BC
:107B30009D028F5F80939D0280919C028F5F809356
:107B40009C02833010F010929C021F9108950F93B5
:107B50001F93CF93DF938C010E94FB17EC010097DA
:107B600031F482E061E472E10E94CF1718C000D0C6
:107B700000D00F92EDB7FEB7319682E0ADB7BEB739
:107B800011968C938DE392E192838183D483C38396
:107B90000E9475170F900F900F900F900F90011586
:107BA000110521F082E0B8010E94CF17CE01DF91CC
:107BB000CF911F910F9108950F931F93CF93DF9350
:107BC0008C010E94F817EC010115110521F002301B
:107BD0001105D9F518C080E090E00E94A73D892BDF
:107BE000A1F181E060E00E9407168AA19BA1892B88
:107BF00011F081E001C082E00E940725BC0182E013
:107C00000E94CF1722C08A819B81892BF1F4888141
:107C10009981892BD1F08AA19BA1892BB1F081E0B8
:107C200060E00E94071683E00E940725BC0182E005
:107C30000E94CF1784EF91E00E948E128AA19BA12F
:107C40000E94FF2B1BA21AA21CA280E090E0DF91F1
:107C5000CF911F910F9108950F931F93CF93DF93AF
:107C6000EB018230910509F4A1C0833091053CF409
:107C7000009709F43EC0019709F0D4C00CC08430CD
:107C8000910509F444C0843091050CF488C005972F
:107C900009F0C8C061C00E94F817FC018081918181
:107CA000892B09F4BFC09F012C5D3F4FAE014B5E95
:107CB0005F4FDE011A9660E217C0F90180818823C8
:107CC00059F0E7E4F2E19491981721F03196992365
:107CD000D1F702C08C9301C06C93F9018081882395
:107CE00011F02F5F3F4F1196A417B50730F31C9288
:107CF00099C080E090E00E94A73D81E060E00E9492
:107D000007162A9682E0BE010E9464178BC0898103
:107D1000A82FB0E0FB01EA0FFB1F228547E452E1E8
:107D2000FA0180E09491921731F03196992311F085
:107D30008F5FF8CF8FEF8F5FE82FFF27E7FDF0957C
:107D4000E95BFD4E8491882311F4FA018491AC0F14
:107D5000BD1F1A968C9366C08981A82FB0E0FB01E5
:107D6000EA0FFB1F2285E7E4F2E180E0949192178D
:107D700029F03196992339F08F5FF8CF882319F0D5
:107D8000E82FE15001C0EFE2FF27E7FDF095E95B46
:107D9000FD4EE491AC0FBD1F1A96EC9343C083E0F7
:107DA00090E04AE050E00E94BC313CC00E94F817CD
:107DB0008C01FC0182819381892BA1F58A81882322
:107DC00049F489E08B8381E0888F19821F8A8A8336
:107DD0008E8B28C089818F5F89838F8B8B3010F1C8
:107DE0001B821A821E8A98012C5D3F4FD901FE0129
:107DF0003A968CE001900D928150E1F7F80182A152
:107E000093A160817181009721F0458D0E94882C9B
:107E100006C0CB01F801658DA9010E943F2DF80134
:107E200093A382A380E090E0DF91CF911F910F9107
:107E300008956F927F928F929F92AF92BF92DF923E
:107E4000EF92FF920F931F93CF93DF93EC017B018F
:107E50000E94F8178C01C230D10509F47EC0C330EE
:107E6000D10534F4209719F1219709F0E5C005C038
:107E7000C630D1050CF0E0C031C0FC01258D922F39
:107E80009370848D86FF04C0992329F494E003C085
:107E9000992309F491E0269526952370235083E0D9
:107EA000989FC0011124280FF7012183C5C081E0EC
:107EB00060E00E9407168CED92E10E94A73D892B9D
:107EC00009F4BAC0F70161818AE0689FB00111240A
:107ED00068587D4E82E00E94CF17AEC0FC01848DB1
:107EE00086FD03C049E050E002C04AE050E0CE0108
:107EF000B7010E94BC31F801808191818F3F9105CB
:107F0000B9F0B0F0F7018181882311F486E0818314
:107F1000F801848D86FD06C0F7018181863010F45A
:107F200088E08183F7018181863010F489E08183C4
:107F3000F801808191818050984208F47DC0F7015A
:107F40008181882311F489E08183F701818189305F
:107F500008F072C089E081836FC0FC018281938147
:107F6000892B09F069C0F7018281882309F45CC07C
:107F7000F801608071806114710409F45DC0858D21
:107F80000E94E117EC01F7014181842F63E00E9418
:107F9000034C292F30E0220F331F220F331F842F71
:107FA0000E94034CD82ED394D22AF4E0DF1609F4B1
:107FB000DD24F80182A093A08D2D0E94E117F80125
:107FC000268D422F50E04F775070BC01649FC00156
:107FD000659F900D749F900D1124BE010E940F4C5F
:107FE0002078262B268FE7012A96F4E2AF2EB12CBB
:107FF000A00EB11ECE01B5010E943C4CC3016D2DF7
:108000000E94A04B8114910459F0F80160817181A4
:10801000C401458D9E010E94882CF80193A382A380
:10802000C501BE010E943C4C90E0F701828188238B
:1080300009F491E0F701928380E090E0DF91CF9125
:108040001F910F91FF90EF90DF90BF90AF909F90A6
:108050008F907F906F900895AF92BF92CF92DF92F2
:10806000EF92FF920F931F93DF93CF930F92CDB7B1
:10807000DEB77B018230910509F46CC08330910535
:1080800034F40097F1F0019709F0DFC00CC08430A0
:10809000910509F449C0843091050CF454C005974A
:1080A00009F0D3C047C09B01265F3F4FC90160E282
:1080B00070E04BE050E00E94354CD70155961C9281
:1080C000C4C0FB018281882309F4BFC08181882359
:1080D00009F4BBC08B01065F1F4F90E060E070E0C9
:1080E000A8010E94492D00D000D00F92EDB7FEB735
:1080F000319622E0ADB7BEB711962C932FED32E149
:1081000032832183948383830E9475170F900F908D
:108110000F900F900F9081E060E00E94071682E0C0
:10812000B8010E94641791C0FB01818190E00E9418
:10813000842C05C0FB01818190E00E94802CD70136
:1081400011968C9382C083E090E040E050E00E9462
:10815000BC317BC090E0FB018281882309F491E06F
:10816000D70112969C930E94F8178C01F701828127
:10817000882371F0D80192968D919C9193970097E6
:1081800029F480E090E00E94842CF70181835DC097
:10819000BAE0AB2EB12CAE0CBF1CD70111968C915E
:1081A00090E0BE016F5F7F4FA5010E94492D6C01D9
:1081B000F801848D82FF08C0C601A0E0B0E0808F86
:1081C000918FA28FB38F3EC0D8018D919C91119752
:1081D000009721F015969C938E931497F8011386BF
:1081E000128613821282D80116961D921D921D923C
:1081F0001C92199711961C921E925C968C915C971A
:108200008C7F5C968C938FEFB6010E94EF25F8016E
:1082100080819181892B21F0C60169810E94A04B48
:10822000D8018D919C91892B69F0C8018496B50184
:108230000E943C4CF7018181D80192968C939297D1
:1082400093961C922FEF3FEF02C020E030E0C9016F
:108250000F90CF91DF911F910F91FF90EF90DF90E2
:10826000CF90BF90AF9008950F931F93CF93DF935C
:10827000EC018B01009731F097FD40C00297029707
:10828000E8F536C081E060E00E940716D80112963A
:108290008C91882359F482E065EF72E10E94CF1738
:1082A00082E06FEE72E10E94CF1722C00E9441254A
:1082B000EDB7FEB737970FB6F894FEBF0FBEEDBF10
:1082C000319622E0ADB7BEB711962C9323EE32E182
:1082D0003283218363837483858396830E94751719
:1082E000EDB7FEB737960FB6F894FEBF0FBEEDBFE1
:1082F000CE01B80140E050E00E94BC3180E090E047
:10830000DF91CF911F910F910895CF93DF93EB01F0
:108310008230910509F44AC08330910534F4009706
:1083200099F0019709F056C005C0863091050CF010
:1083300051C037C00E943725DC0114968C9163E050
:108340000E94034C898346C081E060E00E940716CA
:10835000998183E0989F802D11240E94841582E0EA
:1083600090E00E948E1281B763E00E94034C8983E3
:1083700000D000D00F92EDB7FEB7319692E0ADB7C6
:10838000BEB711969C932EEF32E132832183838313
:1083900014820E9475170F900F900F900F900F90FE
:1083A00019C04FEE5FEF0E94BC3114C08A81882350
:1083B00059F00E943725298143E0249F9001112420
:1083C000FC0124830E941A2690E08A81882309F404
:1083D00091E09A8380E090E0DF91CF910895CF9370
:1083E000DF93EB0182309105C9F1833091053CF4B4
:1083F000009751F08130910509F058C029C08630AE
:1084000091050CF053C024C08A81882309F44EC022
:1084100080E061E00E9407168981845F0E94AE249B
:10842000BC0182E00E94CF1781E060E00E94071645
:108430006981623020F08AE10E94072504C0862FFE
:10844000805F0E94AE24BC0182E00E94CF172EC044
:10845000BE0142E050E00E94BC3128C08A818823DE
:1084600019F18981823018F48E5F89831FC081E001
:1084700060E00E9407168981833051F487E10E94F1
:108480000725BC0182E00E94CF170E94E24509C087
:1084900088E10E940725BC0182E00E94CF170E945C
:1084A000C2452FEF3FEF04C081E08A8320E030E037
:1084B000C901DF91CF910895CF92DF92EF92FF92A1
:1084C0000F931F93CF93DF937C01162F0E94FB1510
:1084D0000E9437256C01173208F06AC0C12FD0E026
:1084E0008E01000F111F000F111F0C0F1D1F0F5EBB
:1084F0001E4FD70112968C91882311F080E001C0A5
:1085000081E00E94C415F6018581843059F08530E0
:1085100089F0BE0124E0660F771F2A95E1F78130CC
:10852000B1F412C094E0CC0FDD1F9A95E1F7C45F5F
:10853000DC4E07C084E0CC0FDD1F8A95E1F7C458FC
:10854000DA4E82E0BE0106C06452784E02C0645C1E
:10855000754E82E00E94CF17D70112968C91882326
:1085600089F4F801848187FD0DC081E060E00E94FC
:108570000716D80114968C910E940725BC0182E051
:108580000E94CF17D8011296ED91FC911397309766
:1085900021F080E090E0B7010995F70186898823F2
:1085A00029F0808D67890E94AB1602C00E940316D5
:1085B000DF91CF911F910F91FF90EF90DF90CF90BF
:1085C00008952F923F924F925F926F927F928F9277
:1085D0009F92AF92BF92CF92DF92EF92FF920F9352
:1085E0001F93DF93CF93CDB7DEB76B970FB6F89499
:1085F000DEBF0FBECDBFD82E45E2481708F45CC2DF
:10860000DE0111968BE1FD0111928A95E9F7A8959B
:108610008D2D90E0FC01EE0FFF1FEE0FFF1FE80F06
:10862000F91FEF5EFE4F0280F381E02D309721F0BD
:1086300081E090E0BD0109958E010F5F1F4FC801D9
:108640006D2D0E945C420E94F8174C0158018EEF7C
:10865000682E8FEF782E0FEF402E0FE7502E1BE085
:10866000212E312C2C0E3D1EF5E0DF9E80011124C1
:10867000B1E1EB2EB1E0FB2EE00EF11E0E947B0E6D
:108680000E945B149C018B30910509F4D1C08C30A1
:1086900091058CF48A3091050CF02DC18130910543
:1086A0000CF04BC14FEF8F3F940709F4F6C10097D0
:1086B00009F433C1E3CF8731910509F4B9C088319A
:1086C000910544F48531910509F4CAC186319105BB
:1086D000A9F6CFC18A31910509F450C082329105C3
:1086E00009F4E5C18931910549F68B81882369F048
:1086F000D7011296ED91FC911397309719F084E011
:1087000090E0ABC18A818F5F48C01F8AF801EF5E9D
:10871000FE4F1081A5E0EA2EF12CEE0EFF1ED39441
:108720000E94F817FC01848D86FD0AC0F2E0DF1676
:1087300039F485E090E0E80EF91EF3E0DF2E03C087
:1087400095E29D152CF0D7018C91811709F45EC03C
:10875000A1E1B1E060E0E12FFF27E7FDF0958C910A
:1087600090E08E179F0711F4D62E50C06F5F6632CF
:1087700011F01596F4CFDD24DA9448C08B8188235C
:1087800071F0D7011296ED91FC911397309719F083
:1087900085E090E062C18A8181508A8388C11F8A06
:1087A0000F5E1E4FF801C080EBEFEE2EEFEFFE2EB6
:1087B000E00EF11EDA940E94F817DC015C968C91B1
:1087C00086FD0BC0B2E0DB1641F47801E6EFFFEF67
:1087D000EE0EFF1EDD24D39402C0D7FC04C0D701E7
:1087E0008C918C1599F0EAECF1E075E2D72E2C2DE6
:1087F000332727FD3095808190E08217930731F071
:10880000DA94BFEFDB1611F03597F5CF8D2D90E0A0
:10881000FC01EE0FFF1FEE0FFF1FE80FF91FEF5EC9
:10882000FE4F0280F381E02D309709F05AC03FC11E
:10883000F70191819923E9F1A92FB0E0FD01E256FA
:10884000FD4F80811816BCF0E1E1F1E020E0492FF6
:10885000552747FD5095808190E08417950711F4C6
:10886000822F06C02F5F263211F03596F4CF8FEF9E
:10887000A256BD4F8C93D7011196EC91F0E0E256D1
:10888000FD4F80810E94E142282F332727FD30953C
:10889000F7018181E82FF0E0E256FD4FC90137FF73
:1088A00004C088279927821B930B808337FFFFC062
:1088B0000DC0D7011296ED91FC9113973097A1F05E
:1088C00082E090E0B501099597FF02C0D194F5C010
:1088D0008B81882309F0EBC0D7011296ED91FC91B2
:1088E000139781E090E0B9C090E08B81882309F470
:1088F00091E09B83DCC08B81882309F4DEC0D70123
:108900001296ED91FC911397309729F083E090E057
:10891000B5010995DDCF1B82CAC08C81813009F475
:10892000A3CE883051F481E00E9458488A810E9489
:10893000A04880E00E945848BAC08C81853009F474
:1089400061C0863070F4823041F1833020F4813090
:1089500009F0ADC012C0833081F0843009F0A7C0A7
:108960004EC0873009F463C0873008F45AC088309D
:1089700021F0893009F09BC060C08F819885892BD8
:1089800011F458864F828F819885821793070CF4D3
:108990008EC01E821D8282E08C838D819E818C011F
:1089A00053E0000F111F5A95E1F7880F991F080F28
:1089B000191F020F131FF401848D86FD15C0F7E700
:1089C000013A1F0789F482E00E94744B81E060E065
:1089D0000E94071682E068E971E10E94CF1784EFD8
:1089E00091E00E948E1202C017FD61C08F819885B0
:1089F000801791070CF45BC01E830D8358C0198645
:108A000045E04C838985AAE08A9FC0011124820F2A
:108A1000931F8F3F910509F008F489877B8E6A8E3A
:108A200046C0283031050CF042C02A8740C02230B1
:108A30003105ECF53B8F2A8F3AC08A81F101E80FAE
:108A4000F11D822F805D8083D7011296ED91FC91FC
:108A50001397309761F182E090E0B501099527C046
:108A600080E00E94480F80E060E240E00E940A2718
:108A70001EC0D7011296ED91FC911397309721F00B
:108A800086E090E0B5010995F7018081882379F4AB
:108A900083E290E00E94412010C08C81883009F070
:108AA000E3CD80E090E0B5010E94A23CDDCDC501A0
:108AB0006D2D0E945C42D8CDDD248D2D6B960FB6B6
:108AC000F894DEBF0FBECDBFCF91DF911F910F9104
:108AD000FF90EF90DF90CF90BF90AF909F908F90DE
:108AE0007F906F905F904F903F902F9008951F93CD
:108AF000182F0E944B25803809F442C080E060E3C3
:108B000072E00E94E81681E068E272E00E94E816D6
:108B100080919E02863210F010929E0217FD04C0D2
:108B2000812F0E94E1420EC080919E020E94E1428C
:108B3000992787FD909597FF03C0909581959F4F4A
:108B400080939E0280E06CE171E00E94E81681E073
:108B500060E671E00E94E81684E068E871E00E9437
:108B6000E81685E060E971E00E94E81686E068E9B1
:108B700071E00E94E81687E060EA71E00E94E81662
:108B80001F910895DF93CF9300D000D000D0CDB7D0
:108B9000DEB7FE01319686E0DF011D928A95E9F786
:108BA00088E089831A8284E2BF014FE859E40E9479
:108BB000882726960FB6F894DEBF0FBECDBFCF91A3
:108BC000DF910895DF93CF9300D000D000D0CDB7D0
:108BD000DEB7FE01319686E0DF011D928A95E9F746
:108BE00088E0898381E08A8384E2BF014FE859E409
:108BF0000E94882726960FB6F894DEBF0FBECDBF21
:108C0000CF91DF910895DF92EF92FF920F931F9320
:108C1000DF93CF9300D000D000D0CDB7DEB7D82EF1
:108C20008E010F5F1F4F86E0F80111928A95E9F7D8
:108C300082E089831A8287E08B838FE9E82E89E4BA
:108C4000F82E84E2B801A7010E94882781E0898379
:108C50001A82DB8284E2B801A7010E948827269647
:108C60000FB6F894DEBF0FBECDBFCF91DF911F913D
:108C70000F91FF90EF90DF900895DF93CF9300D096
:108C800000D000D0CDB7DEB7FE01319686E0DF011F
:108C90001D928A95E9F7198284E2BF014FE959E4F0
:108CA0000E94882726960FB6F894DEBF0FBECDBF70
:108CB000CF91DF9108950F93DF93CF9300D000D031
:108CC00000D0CDB7DEB7542F46E14983482F4F7708
:108CD0004A83880F892F881F990B91958F778B83F3
:108CE000822F8F778C83220F232F221F330B3195F6
:108CF00027702D83802F8F778E8307FF02C0286017
:108D00002D83862F90E08370907024E0880F991F48
:108D10002A95E1F79D81982B9D83552311F090644E
:108D20009D8384E2BE016F5F7F4F4FEA59E40E944A
:108D3000882726960FB6F894DEBF0FBECDBFCF9121
:108D4000DF910F910895DF93CF9300D000D000D032
:108D5000CDB7DEB7FE01319696E0DF011D929A9500
:108D6000E9F794E19983982F9F779A83881F882742
:108D7000881F8B8384E2BF014FEA59E40E94882751
:108D800026960FB6F894DEBF0FBECDBFCF91DF9110
:108D90000895DF93CF9300D000D000D0CDB7DEB7D9
:108DA000FE01319696E0DF011D929A95E9F78983DD
:108DB000862F8F778A83660F672F661F770B7195D3
:108DC0006F776B83842F8F778C83441F4427441FD6
:108DD0004D8384E2BF014FEA59E40E94882726961A
:108DE0000FB6F894DEBF0FBECDBFCF91DF910895CF
:108DF0009C01462F83E1B9010E94C94608959C0158
:108E0000462F8DE0B9010E94C9460895DF93CF93A4
:108E100000D000D000D0CDB7DEB7FE01319696E08D
:108E2000DF011D929A95E9F78983862F8F778A83D0
:108E3000660F672F661F770B71956F776B8384E2E0
:108E4000BF014FEA59E40E94882726960FB6F8948E
:108E5000DEBF0FBECDBFCF91DF910895BC0182E18F
:108E60000E9406470895BC018CE00E9406470895C1
:108E7000DF93CF9300D000D000D0CDB7DEB7FE0196
:108E8000319696E0DF011D929A95E9F791E1998379
:108E90008F708A83862F8F778B83661F6627661F66
:108EA0006C8384E2BF014FEA59E40E94882726962A
:108EB0000FB6F894DEBF0FBECDBFCF91DF910895FE
:108EC000DF93CF9300D000D000D0CDB7DEB7FE0146
:108ED000319696E0DF011D929A95E9F790E199832A
:108EE0008F708A8384E2BF014FEA59E40E94882789
:108EF00026960FB6F894DEBF0FBECDBFCF91DF919F
:108F00000895DF93CF9300D000D000D0CDB7DEB767
:108F1000FE01319626E0DF011D922A95E9F72FE048
:108F20002983282F2F772A83880F892F881F990B51
:108F300091958F778B8367706C831D82442311F02A
:108F400081E08D8384E2BE016F5F7F4F4FEA59E479
:108F50000E94882726960FB6F894DEBF0FBECDBFBD
:108F6000CF91DF910895DF93CF9300D000D000D050
:108F7000CDB7DEB7FE01319626E0DF011D922A95BE
:108F8000E9F72EE02983282F2F772A83880F892F4E
:108F9000881F990B91958F778B8367706C8384E220
:108FA000BF014FEA59E40E94882726960FB6F8942D
:108FB000DEBF0FBECDBFCF91DF910895DF93CF937A
:108FC00000D000D000D0CDB7DEB7FE01319696E0DC
:108FD000DF011D929A95E9F797E099839FE79A83BD
:108FE0009B838F778C8384E2BF0141ED59E40E941B
:108FF000882726960FB6F894DEBF0FBECDBFCF915F
:10900000DF910895DF93CF9300D000D000D0CDB78B
:10901000DEB7FE01319626E0DF011D922A95E9F7C1
:1090200027E02983282F2F772A83880F892F881FED
:10903000990B91958F778B836F776C8384E2BF0157
:1090400041ED59E40E94882726960FB6F894DEBFBA
:109050000FBECDBFCF91DF910895DF93CF9300D0A6
:1090600000D000D0CDB7DEB7FE01319626E0DF019B
:109070001D922A95E9F727E02983282F2F772A8345
:10908000880F892F881F990B91958F778B838FE796
:109090008C8384E2BF0141ED59E40E948827269623
:1090A0000FB6F894DEBF0FBECDBFCF91DF9108950C
:1090B000DF93CF9300D000D000D0CDB7DEB7FE0154
:1090C000319696E0DF011D929A95E9F7882311F415
:1090D00082E001C081E0898380E48A8384E2BE016A
:1090E0006F5F7F4F41EE59E40E94882726960FB6A6
:1090F000F894DEBF0FBECDBFCF91DF910895DF930F
:10910000CF9300D000D000D0CDB7DEB796E0FE01FF
:109110003196DF01292F1D922A95E9F799838F77E0
:109120008A8384E2BF0141EF59E40E948827269692
:109130000FB6F894DEBF0FBECDBFCF91DF9108957B
:10914000DF93CF9300D000D000D0CDB7DEB7FE01C3
:10915000319696E0DF011D929A95E9F795E09983A3
:109160008F778A8384E2BF0141EF59E40E94882708
:1091700026960FB6F894DEBF0FBECDBFCF91DF911C
:109180000895DF93CF9300D000D000D0CDB7DEB7E5
:10919000FE01319696E0DF011D929A95E9F794E081
:1091A00099838F778A8384E2BF0147E15AE40E9462
:1091B000882726960FB6F894DEBF0FBECDBFCF919D
:1091C000DF910895DF93CF9300D000D000D0CDB7CA
:1091D000DEB7FE01319686E0DF011D928A95E9F740
:1091E00084E089838FE78A8384E2BF0147E15AE400
:1091F0000E94882726960FB6F894DEBF0FBECDBF1B
:10920000CF91DF910895DF93CF9300D000D000D0AD
:10921000CDB7DEB7FE01319696E0DF011D929A953B
:10922000E9F793E0998391E09A83982F9F779B8346
:10923000881F8827881F8C8384E2BF0147E25AE495
:109240000E94882726960FB6F894DEBF0FBECDBFCA
:10925000CF91DF910895DF93CF9300D000D000D05D
:10926000CDB7DEB7FE01319686E0DF011D928A950B
:10927000E9F783E089831A8284E2BF0147E25AE476
:109280000E94882726960FB6F894DEBF0FBECDBF8A
:10929000CF91DF910895DF93CF9300D000D000D01D
:1092A000CDB7DEB784E068EF71E00E94E81685E094
:1092B00060E072E00E94E81689E69DE368EC70E0E9
:1092C0000E944C15FE01319686E0DF011D928A95C1
:1092D000E9F78BE0898384E2BF014FE759E40E94FC
:1092E0008827892B19F40E947B0EFDCF26960FB696
:1092F000F894DEBF0FBECDBFCF91DF910895FC0182
:109300008181843219F482818B3021F0CF010E9457
:10931000B226089580E090E00E94F82B0895FC01A9
:109320008181843219F48281883021F0CF010E943A
:10933000B226089580E090E00E94F82B0895FC0189
:109340008181843219F48281882321F0CF010E9427
:10935000B2260895848190E00E94F82B0895FC01C4
:109360008181843219F48281853121F0CF010E94FC
:10937000B2260895438150E0848190E09695982F1D
:109380008827979587956581362F3295330F330F50
:10939000307C20E0822B932B842B952B0E94F82B82
:1093A0000895FC018181843219F48281873021F093
:1093B000CF010E94B2260895858190E00E94F82B8B
:1093C0000895FC018181843219F48281882321F07F
:1093D000CF010E94B2260895838190E00E94F82B6D
:1093E0000895FC018181843219F48281853021F055
:1093F000CF010E94B2260895238130E02F7730708C
:109400004581942F9295990F990F907C80E0822B43
:10941000932B248130E02F7730703695322F22271E
:1094200037952795822B932B0E94F82B0895FC01EA
:109430008181843219F48281843021F0CF010E942D
:10944000B2260895838190E00E94F82B0895FC01D4
:109450008181843219F48281833021F0CF010E940E
:10946000B22608958481881F8827881F9381892BBD
:1094700090E00E94F82B0895DF93CF93CDB7DEB72D
:109480002A970FB6F894DEBF0FBECDBFFE0135960A
:1094900026E0DF011D922A95E9F729E02D83282F88
:1094A0002F772E83880F892F881F990B91958F779F
:1094B0008F8384E2BF0148E75AE49E012F5F3F4F4C
:1094C0000E942527892B29F020E030E040E050E081
:1094D00004C029813A814B815C81B901CA012A9675
:1094E0000FB6F894DEBF0FBECDBFCF91DF910895C8
:1094F000DF93CF9300D000D0CDB7DEB7FC018181E0
:10950000843229F46281862F8950823020F0CF0185
:109510000E94B22682C0838190E0A0E0B0E0248166
:1095200030E040E050E077E0220F331F441F551F2A
:109530007A95D1F7282B392B4A2B5B2B858190E02C
:10954000A0E0B0E07EE0880F991FAA1FBB1F7A95AC
:10955000D1F7282B392B4A2B5B2B868190E0A0E09A
:10956000B0E075E1880F991FAA1FBB1F7A95D1F74C
:10957000282B392B4A2B5B2B878190E0A0E0B0E0B1
:109580007CE1880F991FAA1FBB1F7A95D1F7282B62
:10959000392B4A2B5B2B29833A834B835C836A30BC
:1095A00059F581E060E00E9407168DB79EB70797D6
:1095B0000FB6F8949EBF0FBE8DBFEDB7FEB73196C4
:1095C00082E0ADB7BEB711968C938CE99CE1928393
:1095D000818389819A81AB81BC8183839483A583B4
:1095E000B6830E9475178DB79EB707960FB6F8948D
:1095F0009EBF0FBE8DBF11C021153105410551051C
:1096000019F080E090E002C08FEF9FEFBE016F5F26
:109610007F4F44E050E00E94E02B0F900F900F909E
:109620000F90CF91DF9108951F93DF93CF9300D0D8
:1096300000D000D0CDB7DEB7182F813021F08430B4
:1096400011F08830B9F4FE01319686E0DF011D92F9
:109650008A95E9F7198284E2BF0141EE59E40E943C
:10966000882740E0212F30E028233923232B29F0BD
:1096700041E003C00E943A25482F842F26960FB65A
:10968000F894DEBF0FBECDBFCF91DF911F9108953B
:10969000DF93CF9300D000D000D0CDB7DEB7982FA6
:1096A000813031F0843021F0883011F0823089F43B
:1096B000FE01319686E0DF011D928A95E9F782E08E
:1096C00089839A8384E2BF0141EE59E40E9488278E
:1096D00002C00E94322626960FB6F894DEBF0FBE57
:1096E000CDBFCF91DF910895DF93CF9300D000D00D
:1096F00000D0CDB7DEB7982F813031F0843021F023
:10970000883011F0823089F4FE01319686E0DF0165
:109710001D928A95E9F781E089839A8384E2BF01EB
:1097200041EE59E40E94882702C00E943B262696FB
:109730000FB6F894DEBF0FBECDBFCF91DF91089575
:109740000F931F93DF93CF9300D000D000D0CDB7FD
:10975000DEB78C01FE01319686E0DF011D928A950D
:10976000E9F7802F8F778983C801880F892F881F99
:10977000990B91958F778A836F776B838FEF64E076
:10978000AF010E94F42681E060E00E94071680E0AD
:109790000E940725BC0182E00E94CF1780E090E084
:1097A00060E040E050E00E94EF1A8FEFB8010E94A5
:1097B000EF2526960FB6F894DEBF0FBECDBFCF9132
:1097C000DF911F910F910895629FD001739FF00167
:1097D000829FE00DF11D649FE00DF11D929FF00D41
:1097E000839FF00D749FF00D659FF00D9927729F78
:1097F000B00DE11DF91F639FB00DE11DF91FBD0103
:10980000CF0111240895991B79E004C0991F961780
:1098100008F0961B881F7A95C9F780950895AA1BB2
:10982000BB1B51E107C0AA1FBB1FA617B70710F04B
:10983000A61BB70B881F991F5A95A9F7809590957D
:10984000BC01CD010895FC0105900020E9F7809549
:1098500090958E0F9F1F0895FB01DC0102C00190BF
:109860000D9241505040D8F70895DC0101C06D932E
:1098700041505040E0F70895FB01DC0101900D924A
:109880000020E1F70895AEE0B0E0E9E4FCE40C94D8
:109890002B4F8C0186E08C831A8309838FEF9FE71F
:1098A0009E838D83CE0101960E947B4CEF81F885CB
:1098B000E00FF11F10822E96E4E00C94474FAEE0CB
:1098C000B0E0E5E6FCE40C942B4F8C018EE08C8339
:1098D0001A8309838FEF9FE79E838D83CE010196C4
:1098E0000E947B4CEF81F885E00FF11F10822E96CD
:1098F000E4E00C94474FABE0B0E0E1E8FCE40C940A
:109900001D4F3C012B015A01FC01178216828381F5
:1099100081FD03C06FEF7FEFC6C19AE0892E1E0163
:109920000894211C311CF3012381F20123FD859150
:1099300023FF81912F01882309F4B2C1853239F4C4
:1099400023FD859123FF81912F01853229F490E039
:10995000B3010E94934EE7CF982FFF24EE24992461
:10996000FFE1FF15D0F09B3269F09C3228F4903271
:1099700059F0933291F40EC09D3249F0903369F45E
:1099800041E024C052E0F52A84E0F82A28C098E09B
:10999000F92A25C0E0E1FE2A22C0F7FC29C0892F60
:1099A00080538A3070F4F6FE05C0989C902C1124E8
:1099B000980E15C0E89CE02C1124E80EF0E2FF2A76
:1099C0000EC09E3229F4F6FC6BC140E4F42A07C0B5
:1099D0009C3619F450E8F52A02C0983649F4F20191
:1099E00023FD959123FF91912F01992309F0B8CF81
:1099F000892F8554833018F08052833038F444E046
:109A000050E0A40EB51E5FE359830FC0933631F0CA
:109A1000933779F0933509F056C020C0F501808165
:109A2000898342E050E0A40EB51E610101E010E020
:109A300012C0F501C080D180F6FC03C06FEF7FEF4C
:109A400002C0692D70E042E050E0A40EB51EC601D0
:109A50000E94884E8C015FE7F52214C0F501C0809A
:109A6000D180F6FC03C06FEF7FEF02C0692D70E07C
:109A700042E050E0A40EB51EC6010E947D4E8C014E
:109A800050E8F52AF3FE07C01AC080E290E0B30167
:109A90000E94934EEA948E2D90E008171907A8F3C0
:109AA0000EC0F601F7FC8591F7FE81916F0190E001
:109AB000B3010E94934EE110EA9401501040011549
:109AC000110579F7EAC0943611F0993669F5F7FE79
:109AD00008C0F501208131814281538184E090E00A
:109AE0000AC0F501808191819C01442737FD409592
:109AF000542F82E090E0A80EB91E9FE6F92257FF8E
:109B000009C050954095309521953F4F4F4F5F4F7D
:109B1000E0E8FE2ACA01B901A1012AE030E00E9472
:109B2000BF4ED82ED21840C0953729F41F2D1F7E66
:109B30002AE030E01DC01F2D197F9F3661F090375D
:109B400020F4983509F0ACC00FC0903739F0983741
:109B500009F0A6C004C028E030E00AC0106114FD7E
:109B6000146020E130E004C014FD166020E132E012
:109B700017FF08C0F501608171818281938144E003
:109B800050E008C0F50180819181BC0180E090E047
:109B900042E050E0A40EB51EA1010E94BF4ED82E97
:109BA000D2188FE7F82EF122F6FE0BC05EEFF522F9
:109BB000D91438F4F4FE07C0F2FC05C08FEEF82289
:109BC00002C01D2D01C0192DF4FE0DC0FE01ED0DCA
:109BD000F11D8081803319F499EEF92208C01F5FCE
:109BE000F2FE05C003C08F2D867809F01F5F0F2D90
:109BF000F3FC14C0F0FE0FC01E1510F09D2C0BC01E
:109C00009D2C9E0C911A1E2D06C080E290E0B3019F
:109C10000E94934E1F5F1E15C0F304C01E1510F462
:109C2000E11A01C0EE2404FF0FC080E390E0B3010D
:109C30000E94934E02FF1DC001FD03C088E790E023
:109C40000EC088E590E00BC0802F867891F001FF70
:109C500002C08BE201C080E2F7FC8DE290E0B3012C
:109C60000E94934E06C080E390E0B3010E94934EA1
:109C70009A94D914C0F3DA94F101ED0DF11D8081AD
:109C800090E0B3010E94934EDD20A9F706C080E268
:109C900090E0B3010E94934EEA94EE20C1F743CEC8
:109CA000F30166817781CB012B96E2E10C94394F69
:109CB000DC01CB01FC01E199FECF06C0FFBBEEBB8E
:109CC000E09A31960DB20D9241505040B8F7089588
:109CD000E199FECF9FBB8EBBE09A99278DB3089583
:109CE000262FE199FECF9FBB8EBB2DBB0FB6F894FC
:109CF000E29AE19A0FBE01960895FC010590615029
:109D000070400110D8F7809590958E0F9F1F089591
:109D1000FC016150704001900110D8F7809590953A
:109D20008E0F9F1F08950F931F93CF93DF938C0186
:109D3000EB018B8181FF1BC082FF0DC02E813F8113
:109D40008C819D812817390764F4E881F98101939A
:109D5000F983E88306C0E885F985802F0995892B6A
:109D600031F48E819F8101969F838E8302C00FEF15
:109D70001FEFC801DF91CF911F910F910895FA0154
:109D8000AA27283051F1203181F1E8946F936E7F3A
:109D90006E5F7F4F8F4F9F4FAF4FB1E03ED0B4E02B
:109DA0003CD0670F781F891F9A1FA11D680F791F6C
:109DB0008A1F911DA11D6A0F711D811D911DA11D7D
:109DC00020D009F468943F912AE0269F112430198D
:109DD000305D3193DEF6CF010895462F4770405D28
:109DE0004193B3E00FD0C9F7F6CF462F4F70405DD7
:109DF0004A3318F0495D31FD4052419302D0A9F732
:109E0000EACFB4E0A6959795879577956795BA952B
:109E1000C9F700976105710508959B01AC010A2EF1
:109E200006945795479537952795BA95C9F7620FC8
:109E3000731F841F951FA01D08952F923F924F926C
:109E40005F926F927F928F929F92AF92BF92CF92CA
:109E5000DF92EF92FF920F931F93CF93DF93CDB7D3
:109E6000DEB7CA1BDB0B0FB6F894DEBF0FBECDBF4B
:109E700009942A88398848885F846E847D848C841C
:109E80009B84AA84B984C884DF80EE80FD800C8125
:109E90001B81AA81B981CE0FD11D0FB6F894DEBF08
:0C9EA0000FBECDBFED010895F894FFCF78
:109EAC00FFFFFF2534642D2534643A2000253464EB
:109EBC000000010000FF00020000FF00070000FF8F
:109ECC000000EF41FF00030000FF00008541FF0090
:109EDC00003441FF0000FD31FF01002C40FF010068
:109EEC00193FFF01002C3EFF0100DC3DFF02006A20
:109EFC003AFF0200023CFF0200923BFF0200A33A31
:109F0C00FF0200563AFF0200423AFF02000E3AFFEF
:109F1C0002003838FF0300DF34FF03007E34FF03F8
:109F2C00040000FF0300AE371B03050000220306EC
:109F3C000000220300F536FF0300F036FF03005744
:109F4C0037FF0400FA36FF0400A23CFF0500EB3695
:109F5C00FF05003F36FF0600F035FF06002A35FFEF
:109F6C0006007A34FF06007634FF0700ED32FF005E
:00000001FF
